:10000000F8FF0220990100001D0600007D05000098
:10001000CD050000A5050000F50500005505000010
:100020005505000055050000550500001D0600009F
:100030001D06000055050000D95E00009D5F000010
:100040001D0600001D0600001D0600001D06000024
:100050001D0600001D0600001D0600001D06000014
:100060001D0600001D0600001D0600001D06000004
:100070001D0600001D0600001D0600001D060000F4
:100080001D0600001D0600001D0600001D060000E4
:100090001D0600001D0600001D0600001D060000D4
:1000A0001D0600001D0600001D0600001D060000C4
:1000B0001D0600001D0600001D0600005D4A000030
:1000C0001D0600003D5A00001D060000FD45000011
:1000D0001D060000515900001D0600001D0600000D
:1000E0001D0600001D0600001D0600001D06000084
:1000F0001D0600001D0600001D0600001D06000074
:10010000B9670000CD670000E1670000F5670000F7
:100110001D0600000D4D00001D0600001D0600001C
:100120001D0600001D0600001D0600001D06000043
:100130001D0600001D0600001D0600001D06000033
:10014000B15F00001D060000115C00001D060000EC
:10015000014900001D0600001D0600001D060000EC
:100160001D0600001D0600001D0600001D06000003
:100170001D0600001D0600001D0600001D060000F3
:100180001D0600001D0600001D0600001D060000E3
:100190001D0600001D060000584B4CF2205210B501
:1001A0001A804DF628121A8000BF00BF00F06AFBCB
:1001B000534B4FF030621A60524A9A60524ADA60EA
:1001C000524B4FF470021A60514A136813F4807353
:1001D00001BF50490B604FF4A85313604E4B4F4979
:1001E0001A78100742BF1A7842F008021A704C4B76
:1001F0002A221A704B4A4C4B8B4204D252F8040FFD
:1002000043F8040BF8E7494B494A0021934202D2D4
:1002100043F8041BFAE7474A4748002350F82310E5
:1002200042F823100133662BF8D1444B444A802115
:1002300003F8011B9342FBD1424B3E4A1A60424BEA
:100240008A221A70A3F5805324225A70A0221A70B1
:100250009A799107FCD59A79D206FCD43B4A9379D6
:1002600003F00C03082B394BF9D103221A714022F9
:100270005A719A799406FCD534498A79334B5006E1
:10028000FBD5334A334911600221516020221A7094
:100290009A7902F00C020C2AFAD12F4B2F4A1A60DD
:1002A0002F4B4BF67F321A6000225A60072243F828
:1002B000042C2C4AC3F80C2D62B604F089FA154BB5
:1002C0001B68DA0705D5284804F03EFA274B284A70
:1002D0001A60284B1B785B0609D5244C244B2268F6
:1002E0009A4204D1204804F02FFA0023236006F03C
:1002F0009DFA00F0CDFA04F03BF9FEE70E20054030
:1003000030800440823F04000100002B88ED00E0B3
:1003100010D0034014D0034002D007403490022094
:1003200000E007404C820000F88602203490022052
:1003300000C00220008202200000000000E400E073
:1003400056E400E008ED00E00050064000400640A2
:10035000448004400000131104800440C0100500D4
:1003600014E000E00000202000DD68501CE00340A5
:10037000A5C3945A00F00740FFFFFFFFFFFFFFFFF8
:10038000FFFFFFFFFFFFFFFFFFFFFFFFFFFFFFFF7D
:10039000FFFFFFFFFFFFFFFFFFFFFFFFFFFFFFFF6D
:1003A000FFFFFFFFFFFFFFFFFFFFFFFFFFFFFFFF5D
:1003B000FFFFFFFFFFFFFFFFFFFFFFFFFFFFFFFF4D
:1003C000FFFFFFFFFFFFFFFFFFFFFFFFFFFFFFFF3D
:1003D000FFFFFFFFFFFFFFFFFFFFFFFFFFFFFFFF2D
:1003E000FFFFFFFFFFFFFFFFFFFFFFFFFFFFFFFF1D
:1003F000FFFFFFFFFFFFFFFFFFFFFFFFFFFFFFFF0D
:10040000FFFFFFFFFFFFFFFFFFFFFFFFDEF9FFFF23
:10041000FFFFFFFFFFFFFFFFFFFFFFFFFFFFFFFFEC
:10042000704700BF05F0FEBC00F0CEBB00F0E6BB9D
:1004300000F0F0BB00F01EBD00F04ABD00F0F4BBC0
:1004400000F054BD00F0A5BD00F0DCBC00F0FCBB2A
:1004500000F0E6BC00F0FABC05F040BC05F03EBC84
:1004600000F02EBA00F06EBA00F09CBA02F04EB85E
:1004700002F0E3BA02F023B902F0B5B902F0D6BB3C
:1004800002F03DBD02F0A5BA02F051BC02F086BCFC
:1004900002F08DBC02F0D2BD02F06EBD02F065BE6E
:1004A00002F0A7BC02F0E8BE02F011BF02F0E4BA0D
:1004B00002F0D0BA02F00EBB02F0BDBC02F02FBFBA
:1004C00002F07EBF02F0F2BF01F0FABF03F076B88F
:1004D00003F05EBB03F036BB03F08EBB03F0A9BB99
:1004E00003F0C4BB00F0F7B900F01EBA704700BFBC
:1004F00003F004BC7047FFFF10B5054C237833B9F7
:10050000044B13B10448AFF300800123237010BDE6
:10051000349002200000000050820000084B10B50B
:100520001BB108490848AFF300800848036803B9C5
:1005300010BD074B002BFBD0BDE81040184700BF93
:100540000000000038900220508200003490022009
:1005500000000000084B00221A601EF0040F0CBFC0
:10056000EFF30880EFF309808169DFF8042010477A
:1005700021060000704700BF50900220084B012266
:100580001A601EF0040F0CBFEFF30880EFF3098030
:100590008169DFF80420104721060000704700BF82
:1005A00050900220084B02221A601EF0040F0CBF6C
:1005B000EFF30880EFF309808169DFF8042010472A
:1005C00021060000704700BF50900220084B032214
:1005D0001A601EF0040F0CBFEFF30880EFF30980E0
:1005E0008169DFF80420104721060000704700BF32
:1005F00050900220084B04221A601EF0040F0CBF1A
:10060000EFF30880EFF309808169DFF804201047D9
:1006100021060000704700BF50900220FFF79ABFEC
:100620002DE9F04788B0036800934368019383681D
:100630000293C36803930369049343690593836931
:1006400006930546C3696648079300F0E3FA654BD5
:100650001B68013B032B0BD8DFE803F002040608FC
:10066000614806E0614804E0614802E0614800E05A
:100670006148DFF8F0A1DFF8088200F0CBFA5F48AC
:1006800000F0C8FA00995E4800F0BCFB01995D4893
:1006900000F0B8FB02995C4800F0B4FB03995B489A
:1006A00000F0B0FB04995A4800F0ACFB059959489A
:1006B00000F0A8FB0699584800F0A4FB079957489A
:1006C00000F0A0FB2946564800F09CFB554B5648CD
:1006D000196800F097FB554B5548196800F092FBDC
:1006E000544B5548196800F08DFB544B5448196819
:1006F00000F088FB534B5448196800F083FB534BC0
:100700005348196800F07EFB524B5348196800F0BB
:1007100079FB334800F07EFA504800F07BFAA5F5EB
:10072000007405F5007521464D484E4E00F06AFBF9
:100730004D4800F06FFADAF8003013F4802F01D042
:1007400004F0E4FA04F120092746474504D8397833
:10075000464800F057FB02E0454800F05BFA2020D5
:1007600000F032FA33685B0301D504F0CFFA0137A9
:100770004F45EAD13F4800F04DFA444504D820786F
:10078000A0F120035E2B00D9202000F01DFA336871
:100790005F0301D504F0BAFA01344C45EDD1364877
:1007A00000F038FAA54202D9344B9C42BBD9002351
:1007B00000933368580301D504F0A8FA336859054B
:1007C00001D504F04BF933681A0501D505F036F967
:1007D0003368DB0401D503F011FF009B0133E7E729
:1007E000057E000050900220D4750000DF750000E7
:1007F000E9750000017600000D7600001B76000010
:1008000040760000527600006476000076760000A4
:10081000897600009B760000AD760000BF76000070
:10082000D176000028ED00E0E47600002AED00E03B
:10083000F67600002CED00E00877000030ED00E0D7
:100840001A77000038ED00E02C77000014ED00E08E
:100850003F7700003CED00E0517700006477000036
:1008600075770000348004407A7700007E770000BE
:10087000D67D00008377000086770000DFFF02202E
:10088000FFFF0220014B10221A8070470020054014
:100890007047FFFF094908B50B6868B16A461844FC
:1008A000A2F50052904206D305F0BAFF0C23036074
:1008B0004FF0FF3008BD0860184608BDFC860220D6
:1008C00038B500200425040205F008FA013D40EA8D
:1008D0000400F8D138BD036810B51BB319460C7875
:1008E000202C0B4601F1010201D11146F7E7222C21
:1008F00009D1134611460A4611F8014B222C08D0A3
:10090000002CF8D105E00A460131147814F0DF0F0D
:10091000F9D1117801F0FD01202904BF002102F86E
:10092000011B0260184610BD036807B50BB9002013
:1009300005E001A900F02DFB0028F8D0019803B0D4
:100940005DF804FB08B58378013B0B2B19D8C378FD
:10095000013B1E2B17D80379172B16D843793B2B55
:1009600015D883793B2B14D80389B3F57A7F12D23B
:100970004389B3F57A7F10D2094800F04BF9002083
:1009800008BD012008BD022008BD032008BD0420C9
:1009900008BD052008BD062008BD072008BD00BF12
:1009A0008A77000010B5044686B00A4800F032F994
:1009B0006089049020890390A07902906079019069
:1009C00020790090E378A2782188034800F01AFA91
:1009D00006B010BD8A770000A4770000214B224AA0
:1009E00010B59A61214ADA6102F580225A604FF00F
:1009F00080529A601E4ADA604FF0A0521A6140F6A7
:100A0000FF7200205A610422186012681A620221E3
:100A10005862032209781278090441EA026101222E
:100A200041F0F801147883F8352041EA04219962F5
:100A300083F836200F4983F8372083F8342083F871
:100A4000382083F8392083F83A2083F83B2083F854
:100A50003C0083F83D0083F83E0083F83F00D962F4
:100A6000196310BD008702200000FF1FFFFF030075
:100A7000FFFF0100000E270710B53A483A4C00F07E
:100A8000C9F83A4800F0C6F894F835302BB194E82C
:100A9000060037480A4400F0B5F994F83520324B87
:100AA0002AB19968DA6833480A4400F0ABF994F83F
:100AB00035202D4B2AB119695A692F480A4400F094
:100AC000A1F994F83420284B2AB19969DA692B48A6
:100AD0000A4400F097F994F83A302BB1224B284899
:100AE00093F83B1000F08EF994F83E302BB11E4B7A
:100AF000244893F83F1000F085F994F83C302BB16E
:100B0000194B214893F83D1000F07CF994F83830E7
:100B100013B11E4800F07EF894F8393013B11C4828
:100B200000F078F81B4800F075F8216A1A4800F0C8
:100B300069F9616A194800F065F9A16A184800F07E
:100B400061F9184800F066F8E26A174B1748B2FBE3
:100B5000F3F103FB112200F055F91548BDE81040F0
:100B600000F058B8BC77000000870220D57700005D
:100B7000E877000004780000207800003C7800004E
:100B8000587800007878000098780000B878000065
:100B9000C1780000CA780000D6780000FB78000019
:100BA000207900004579000040420F004C79000098
:100BB000067E0000014800F02DB800BF77790000E4
:100BC000704770477047FFFF0A2810B5044602D1EE
:100BD0000D20FFF7F9FF074A13681BB1591C1C7061
:100BE000116010BD044B1B681BB12046BDE81040CE
:100BF000184710BD54900220A4A0022038B5044C20
:100C0000256820600846FFF7DFFF256038BD00BF7C
:100C1000A4A0022010B5441E14F8010F10B1FFF774
:100C2000D3FFF9E710BDFFFF064B70B51E681860D3
:100C30004D1E1C4615F8010F10B1FFF7C5FFF9E76F
:100C4000266070BDA4A002202DE9F047044688B0BC
:100C50000D462078002800F0D280252801D00134EC
:100C600072E06078302803D1E31CA078012207E00D
:100C70002D280DBFA078A31C0022E31C08BF022270
:100C80002A2803D000271C460A2104E02F68187880
:100C90005C1C043509E0A0F13003092B05D801FBE9
:100CA0000707303F14F8010BF5E700F0DF034C2B8A
:100CB00002BF207842F004020134002800F09F8037
:100CC000602886BFA0F12003DBB203464F2B12D071
:100CD00006D8432B30D0442B3DD0422B38D033E0C4
:100CE000552B38D0582B2CD0532B2DD1D5F8008034
:100CF0002E1D434602E04FF0080E2EE0C8EB030520
:100D000013F8011B0029F9D1900709D4BD4205F160
:100D1000010904D22020FFF757FF4D46F6E74D4664
:100D20004046FFF777FFAF4201D8354691E72020D4
:100D3000FFF74AFF0135F6E728782E1DFFF744FF3D
:100D4000F3E74FF0100E08E0FFF73EFF2E46ECE70A
:100D50004FF0020E01E04FF00A0E442B296805F116
:100D6000040604D10029BCBF494242F01002782891
:100D700014BF4FF007084FF027080020B1FBFEFC1E
:100D80000EFB1C15EBB2092D84BF4344DBB230339C
:100D90006146451C0DF80030BCF1000F04D0202D39
:100DA00001D02846EAE71F20D10605D508AB1D442F
:100DB0002D2305F8203C851C12F0010F14BF4FF0C5
:100DC000300A4FF0200A9307A84609D4B84508F125
:100DD000010904D25046FFF7F7FEC846F6E7C846B9
:100DE000013D1DF80500FFF7EFFE002DF8D1474546
:100DF0009BD92020FFF7E8FE08F10108F7E708B0CB
:100E0000BDE8F0870FB407B504A951F8040B0191B0
:100E1000FFF71AFF03B05DF804EB04B07047FFFF63
:100E20000EB417B505A9084C51F8043B20601846CC
:100E30000191FFF709FF226800231370236003B0BC
:100E4000BDE8104003B07047549002200EB433B593
:100E500005A9074C51F8043B25682060184601910C
:100E6000FFF7F2FE256002B0BDE8304003B07047E6
:100E7000A4A00220154B1A682DE9F04107461E4632
:100E800072B100244D1E07E00D2817D008280AD1A2
:100E900014B1013CFFF798FE336898470028F3D15E
:100EA0000020BDE8F0811F28F6DDAC42F4DA3855A9
:100EB00004F10108FFF788FE4446EDE700233B55A7
:100EC0000A20FFF781FE0120BDE8F081A0A00220EA
:100ED00038B5054C0B462568206011461846FFF7CB
:100EE000C9FF256038BD00BFA0A0022070B5002357
:100EF0000B6002681378202B02D101320260F8E700
:100F00002D2B01BF531C03605378012618BF002608
:100F1000302B19D10268531C03605378622B06D022
:100F2000782B09D1931C03609378102513E0931C50
:100F30000360937802250EE0202B28D9A3F130021C
:100F4000092A07D9002070BDA3F13002092AF9D877
:100F50000A2500E008250024202B15D9602B84BF2A
:100F6000203BDBB2A3F13002D2B2102A03D9373BC7
:100F7000DAB2092AE6D9AA42E4D2036804FB0524BE
:100F80005A1C02605B78E7E706B164420C600120FE
:100F900070BD70B500230B6002681378202B02D15E
:100FA00001320260F8E72D2B01BF531C0360537818
:100FB000012618BF0026302B19D10268531C03608C
:100FC0005378622B06D0782B09D1931C0360937859
:100FD000102513E0931C0360937802250EE0202B6C
:100FE00028D9A3F13002092A07D9002070BDA3F146
:100FF0003002092AF9D80A2500E008250024202B10
:1010000015D9602B84BF203BDBB2A3F13002D2B2F2
:10101000102A03D9373BDAB2092AE6D9AA42E4D228
:10102000036804FB05245A1C02605B78E7E706B1FD
:1010300064420C60012070BD70B506460D46144632
:10104000237863B10820FFF7BFFD2020FFF7BCFD28
:101050000820FFF7B9FD2378013B2370F0E7304605
:10106000FFF7D8FD257070BD2DE9F3471A4D1B4ED3
:101070002C78074656F824008846914608B105F0BA
:1010800005FC08F1010A504605F0F8FB46F824007B
:1010900050B152463946013405F0B8FEE4B2132C83
:1010A0008ABF00232C702B70B9F1000F11D00C4CAB
:1010B000206870B10B4B1B785BB901AB42463946D7
:1010C00001F091FB21680A2002F062FD206801F026
:1010D00080FC02B0BDE8F0875990022064900220A5
:1010E0005C9002206290022070B500240C4D2646D0
:1010F00055F8240018B105F0C9FB45F82460013407
:10110000142CF5D1074C084B206800251D7028B120
:1011100001F093FC206805F0B9FB256070BD00BFAD
:10112000649002205C9002205990022070B5124C0D
:101130009EB00021206801F079FDD0B90125226818
:101140007821684602F0FEFC98B1684605F0D8FFA9
:1011500000280CDD1EAB1844002300F8793C29461A
:101160006E1C6A460548FFF74DFE3546E7E701303D
:10117000E5D11EB070BD00BF5C900220687A00000F
:101180002DE9F0431D4C9FB0074689462068002199
:10119000904601F04BFD60BB012506462268782190
:1011A000684602F0CFFC78B1684605F0A9FF002838
:1011B00005F1010504DD1EAB184400F8796C01E06F
:1011C000013001D0A845E9D12068C16801F02EFDA9
:1011D00010B10B48FFF71EFDA8450AD169463846F5
:1011E00005F012FF384605F08BFF89F8000000205B
:1011F00000E001201FB0BDE8F08300BF5C9002203A
:10120000727A00002DE9F743074688460090009B5C
:101210001A78202A07D198F800203A44934202D243
:1012200001330093F3E7DFF86490002454F8095089
:10123000009E284605F064FF31460246284605F028
:10124000CDFFD0B909EB04031D79012D02D0022D89
:1012500003D012E0FFF76AFF13E0013601A96846E8
:101260000096FFF743FE40B1019A4146013A3846E5
:10127000FFF786FF08B9002503E00834182CD5D104
:10128000F9E7284603B0BDE8F08300BF8C79000081
:101290002DE9F04FC34B1D78C34B16461A68A1B019
:1012A00004460F469846002A3DD1DFF81C9399F872
:1012B0000030002B3AD1002E38D0282005F0DEFA7D
:1012C000C8F8000058B31322314601F01FF918B9CD
:1012D000054602AE814616E0B448FFF793FD25E0CF
:1012E00005F00EFF002817DD411E20AB0B44013531
:1012F000EDB20022C9B2304603F8789CFFF7B4FE85
:10130000142D28BF0025D8F800207821304602F09F
:1013100019FC86420AD1E3E70130F4D106E001234B
:1013200089F8003002E00EB9FFF7DEFEDFF88092A8
:101330004FF0000804F0D2FC43B20133FAD09C4BCA
:101340009C4A93F900109C4B93F9003052F833609B
:1013500016F801E0C0B27045DFF85CE27BD013D232
:10136000013B5BB29446002B29DB02EBC30A9AF8DF
:1013700004A0514505DA5CF8336016F801A08245F7
:101380001AD0013B5BB2EEE701335BB2924602E05A
:101390000CF101035BB25FFA83FCBCF1150F0ED8B0
:1013A00002EBC30B9BF804B05945F1DA5AF83360ED
:1013B00016F801B08345EBD18EF800304BE07C4A43
:1013C000002313708EF8003080467C4B1878B842AA
:1013D0009E46AFD07A490A7890428A460BD31A7853
:1013E000501C187004F802800A7897420FDD744987
:1013F00001320A700BE09EF8000052B28242EEDB2E
:10140000A01814F802C080F801C0013AF3E793F87D
:1014100000B00BF1FF3B4FFA8BFB9AF8002093458D
:101420000ADA14F80B0001930BF1010BFFF7CCFB68
:101430004FFA8BFB019BF0E793F900B09AF800306C
:101440009B45BFF677AF08200BF1010BFFF7BCFB04
:101450004FFA8BFBF2E79EF9003002EBC302013139
:10146000137949B2994289F800107FF463AF537938
:10147000514A4FF0000A89F800A082F800A0152B0D
:101480003FF658AF01A252F823F000BFCB13000083
:1014900005150000CD15000069170000E5140000D7
:1014A00035130000451600004F17000069160000B4
:1014B00003170000831600007115000035130000AB
:1014C000CD150000ED150000451600003513000095
:1014D0003513000083160000031700004F170000AB
:1014E00069170000354D84F801A0032323702A46B4
:1014F00000213448FFF7A0FD314B85F800A083F8A8
:1015000000A041E1DFF8B4B09BF80030002B3FF4BD
:1015100011AFDFF8ACA09AF80020013B013A082097
:101520008BF800308AF80020FFF74EFB9BF9003063
:101530009AF80020934209DAE21801935078E054B7
:10154000FFF742FB019B01335BB2F1E72020FFF77D
:101550003BFB9BF900B09AF800309B453FF7EAAEA1
:1015600008200BF1010BFFF72FFB4FFA8BFBF2E783
:10157000134D2B780A2004F803A0FFF725FB29461A
:101580002046FFF73FFE30B9297831B101222046CD
:10159000FFF76AFD01E000232370084A002313705F
:1015A0002B70F1E0599002205C9002209C7A0000A0
:1015B00063900220B87900005890022061900220C8
:1015C00060900220077E000062900220DFF8CCA12C
:1015D0009AF80030002B3FF4ADAE0820FFF7F4FA84
:1015E0009AF80030013B8AF80030F1E76849DFF8EB
:1015F000ACB10A789BF8003093428A463FF49AAE29
:10160000013A0A709AF800205BB2934208DAE218B5
:1016100001935078E054FFF7D7FA019B0133F1E7CB
:101620002020FFF7D1FA9BF900B09AF800309B45D3
:101630003FF780AE08200BF1010BFFF7C5FA4FFA18
:101640008BFBF2E7DFF854A1DFF844B19AF80030E1
:101650009BF800209A427FF66DAE5A1C8AF8002053
:10166000E05CFFF7B1FAF1E7DFF830A149485246F4
:101670000021FFF7E1FC464A00238AF8003013708E
:1016800058E6454BB5B9D3F84CA0BAF1000F11D0CC
:10169000504605F035FD3E4DC2B22870013251462C
:1016A000204605F0B3FB29783C4A2046FFF7C4FCEE
:1016B00013253FE605F1FF3B53F82B1031B10846E7
:1016C0000191DFF8CCA005F01BFD31E0324B53F85F
:1016D00025B0BBF1000F3FF42DAE584605F010FDCC
:1016E000DFF8ACA08AF80000C2B2013259462046A9
:1016F00005F08CFB294A9AF800102046FFF79CFC65
:1017000018E6132DDFF888A0234B08D1D3F800B0DA
:10171000BBF1000F03D0584605F0F2FCE2E705F1FB
:10172000010B53F82B1071B10846019105F0E8FC4C
:10173000C2B28AF8000001320199204605F066FB2A
:101740005FFA8BF5D6E78AF800102170D2E7134ACA
:101750000F491378097899427FF6ECAD591C117046
:10176000E05CFFF731FAE5E5DFF830A09AF80030E9
:10177000002B3FF4DFAD0820FFF726FA9AF800307F
:10178000013B8AF80030D5E5204621B0BDE8F08F56
:1017900060900220077E0000649002206190022089
:1017A00042884378007843EA022340EA03207047E6
:1017B0000B0A017043700B0C090E8370C1707047E7
:1017C000024400F8011B9042FBD1704730B504463B
:1017D00014F8013B11F8015B5B1B151BE84201D0BB
:1017E000002BF5D0184630BD83690239023B99427F
:1017F0003DBF4389C06A01FB030000207047FFFF23
:10180000F0B5056885B12C4614F8013B202B0ED9A4
:101810003A2BF9D12B78303BDAB2092A0AD8AA1C24
:10182000944207D1032B27DD4FF0FF30F0BD144B5E
:101830001878F0BDDFF84CE000235EF823702E46E8
:1018400017F8012B16F8011BA2F1610CBCF1190F5E
:1018500098BF203AA1F1610C98BFD2B2BCF1190F28
:101860009CBF2039C9B22AB19142E9D00133042B7F
:10187000E3D1D9E7B442F9D104601846F0BD00BF06
:10188000B4900220EC7B000038B50D46044678B1D8
:1018900003686BB11A785AB18188DA88914207D10E
:1018A000587802F089F910F0010001D1236801E0B5
:1018B000092000232B6038BD01380A4411F8013B90
:1018C00000F8013F9142F9D17047CA7E8B7E032810
:1018D00043EA022301BF487D0A7D42EA002243EA2F
:1018E000024318467047C2F307238A76CB76037803
:1018F000032B01BF120C0A75120A4A7570470023A8
:1019000070B51A462E25C669541CB25C202A0AD02E
:10191000052A08BFE522092C02BFCE1801337572D3
:10192000CE18013372720B2C2246ECD10B440022EC
:101930005A72C369DB7A0B72C46904F11C00FFF7A9
:101940002FFF0860E27DA37D43EA0223CB80627E05
:10195000237E43EA02238B8070BD70B5C3780446B2
:101960000BB9002070BD00F13406026B40780123F2
:10197000314602F05EF980B9216B636AE269E0707A
:10198000CB1A9342EDD2A378022BEAD10A44012369
:101990003146607802F04DF9E3E7012070BDF8B5FB
:1019A0000446FFF7DAFF0546002842D12378032BCF
:1019B00037D12779012F34D104F1340601464FF491
:1019C00000723046FFF7FCFE552384F83232AA231A
:1019D00084F8333252234122722184F8343084F85F
:1019E0003530612384F8363084F8372084F81A22A1
:1019F00084F81B3284F8181284F8191204F5077061
:101A00002169FFF7D5FEE16804F50870FFF7D0FE05
:101A1000226A6078013222633B46314602F009F9BE
:101A2000257100221146607802F020F9003018BFBD
:101A30000120F8BD036B8B4270B506460D4611D0F0
:101A4000FFF78BFF044670B92A46012306F13401E3
:101A5000707802F0D1F800281CBF4FF0FF35012448
:101A6000356300E00024204670BDFFFF002310B561
:101A7000C3704FF0FF3303630446FFF7DBFF18BB6F
:101A800094F8332294F8323243EA02234AF655227C
:101A900093421BD194F83430EB2B03D01833DBB2D4
:101AA000012B15D803220B4904F16A00FFF78EFEC3
:101AB00078B10522084904F18600FFF787FE002867
:101AC00014BF0220002010BD042010BD032010BD53
:101AD000022010BD0E7B0000127B00002DE9FF41AB
:101AE00000230B600F461546FFF78AFE061EC0F264
:101AF00027819B4B53F82640002C00F023813C604B
:101B0000237805F0FE0583B1607802F055F8C1072F
:101B10000BD4002D00F0188100F0040303F0FF0047
:101B2000002B00F019810A2016E10023F0B2237087
:101B30006070012102F04CF8C20700F107810DB17D
:101B40004307F0D400212046FFF790FF02281FD161
:101B500004F5FD75002115F8040C10B12846FFF7B7
:101B60001FFE4DF821000131042905F11005F2D1C5
:101B700000255DF8256036B131462046FFF776FF37
:101B8000012801D80CE003200135042DF1D1DFE05C
:101B9000042800F0E080012801D90D20DCE00026B7
:101BA00094F8402094F83F3043EA0223B3F5007FD5
:101BB000F3D194F84B5094F84A3053EA052504D1F8
:101BC00004F15800FFF7ECFD054694F84470E56118
:101BD0007B1E012BA770E0D894F841108BB2638173
:101BE000002BDAD04B1E0B42D7D194F8468094F8E4
:101BF000453043EA082818F00F0FA4F80880CCD12C
:101C000094F8480094F8473053EA002003D104F1D7
:101C10005400FFF7C5FD94F8433094F8422052EA8F
:101C20000323BAD005FB07FE03EB1812724490425F
:101C3000B3D3801AB0FBF1F14A484F1E8742ACD8AB
:101C40004FF6F570814206D840F6F577B9428CBF61
:101C50000227012700E00327023133443244032FD7
:101C6000A16126626362E26210D194F85F2094F869
:101C70005E3053EA022390D1B8F1000F8DD104F108
:101C80006000FFF78DFDA062890010E0B8F1000F41
:101C900083D0022F4FEA410018BF4018734418BF89
:101CA00001F00101A3620CBF014601EB500101F2FA
:101CB000FF11B5EB512FFFF470AF4FF0FF332361ED
:101CC000E360032F4FF0800323712FD194F8652038
:101CD00094F8643043EA0223012B27D1711C20467B
:101CE000FFF7A8FE10BB94F8332294F8323220712B
:101CF00043EA02234AF65522934217D104F13400F5
:101D0000FFF74EFD184B984210D104F50670FFF70F
:101D100047FD164B984209D104F50770FFF740FDC7
:101D2000206104F50870FFF73BFDE060104A277062
:101D3000138801339BB200201380E38060610BE0C5
:101D40000B2009E00C2007E0284605E0032003E013
:101D500004287FF422AF012004B0BDE8F08100BF69
:101D6000B8900220F4FFFF0F52526141727241613C
:101D7000B690022001292DE9F04706460C4615468B
:101D80006FD9836999426CD20378022B3CD0032B24
:101D90004CD0012B65D101EB5108416A01EB582170
:101DA000FFF748FE074600285CD106F1340A08F127
:101DB0000109C8F3080814F001041FBF1AF808301D
:101DC00003F00F022B0103F0F00314BF1343EBB237
:101DD0000AF80830716A0123F37001EB592130468B
:101DE000FFF728FE0746E8BBC9F3080914B1C5F39D
:101DF000071506E01AF80910C5F3032521F00F01B5
:101E00000D430AF8095029E0416A01EB1421FFF75C
:101E100011FE074630BB640006F1340304F4FF747E
:101E20001A191D55C5F30725557017E0416A01EBD6
:101E3000D411FFF7FFFD0746A0B9A40006F1340353
:101E400004F4FE741C442046FFF7AAFC25F07045FC
:101E500000F0704129432046FFF7AAFC0123F370EC
:101E600000E002273846BDE8F0870129F8B50546AD
:101E70000C4652D9836999424FD20378022B29D05C
:101E8000032B38D0012B48D101EB5106416A01EBFD
:101E90005621FFF7CFFD10B14FF0FF30F8BD771C92
:101EA000696AC6F308062E4401EB5721284696F8C6
:101EB0003460FFF7BFFD0028EED1C7F308073D44AB
:101EC000E30795F8340046EA00204CBF0009C0F350
:101ED0000B00F8BD416A01EB1421FFF7ABFD0028B0
:101EE000DAD16400343504F4FF742B1958782B5D73
:101EF00043EA0020F8BD416A01EBD411FFF79AFDD7
:101F00000028C9D1A40005F1340004F4FE74204473
:101F1000FFF746FC20F07040F8BD0120F8BDB1F598
:101F2000001FF8B505460C4601D30220F8BDCA06CD
:101F3000FBD182680668296162B93378022B01D926
:101F4000B36A33B93389B3EB541FEED9B36AAB61CB
:101F500016E01A4677897F02BC4211460CD32868E6
:101F6000FFF783FF431C024618D00128DDD9B3696F
:101F70009842DAD2E41BEFE73046FFF735FCA86160
:101F8000AB696A61002BD0D003EB54233436C4F321
:101F900008043444AB61EC610020F8BD0120F8BDB9
:101FA0002DE9F041804605680F4631B9EE68A6B1CB
:101FB000AB699E4228BF012610E02846FFF755FF77
:101FC000012861D9421C03D14FF0FF30BDE8F081F8
:101FD000AB69984259D33E4600E001262B6913B9FC
:101FE0000020BDE8F081BE4217D1AB69D8F80000EF
:101FF000741C9C4228BF02242146FFF736FF0128AB
:1020000042D0431CE0D038B1EB68012B05D9AA6956
:10201000934238BF1E4600E0A4B93446AB69013490
:102020009C4202D3012EDBD902242146D8F80000BD
:10203000FFF71BFF30B1012826D00130C4D0B442D5
:10204000ECD1CDE74FF0FF3221462846FFF792FE54
:10205000C0B947B9AA692B69EC60023A93420AD821
:10206000013B2B6107E0224639462846FFF782FEF6
:102070000028EFD006E02B7943F001032B712046B6
:10208000BDE8F08101289FD00120BDE8F081F8B5BE
:102090000D46012D0746114601D80220F8BD0468FF
:1020A000A3699D42F9D22AB14FF0FF322046FFF7D3
:1020B00061FE08BB29463868FFF7D7FE064608B917
:1020C0000020F8BD0128E8D0431C14D00022294686
:1020D0002046FFF74FFE78B9A2692369911E8B4213
:1020E00005D201332361237943F001032371964222
:1020F0003546DFD3E4E70120F8BDF8B505460E46C6
:10210000FFF72BFC0446F8B931462846FFF76CFB75
:1021100005F13406074628634FF400722146304625
:10212000FFF74EFB6B899C4204D36889001B18BFE4
:102130000120F8BD01233A193146687801F079FD94
:102140000028F2D10134EDE70120F8BD2DE9F84374
:10215000076906682037B7F5001F24BF0023836195
:10216000836904468946002B45D0C7F30808B8F1B7
:10217000000F39D141690133836131B93389B3EB40
:10218000571F31D80023A36135E07389013B13EA5F
:10219000572329D13046FFF768FE0128054602D8AB
:1021A0000220BDE8F883421C02D10120BDE8F8837B
:1021B000B369984212D3B9F1000FE3D061692046A8
:1021C000FFF7EEFE0546C8B10128E9D0431CECD06C
:1021D00001463046FFF791FF0028E6D165612946A8
:1021E0003046FFF701FBA061343646442761E661C3
:1021F0000020BDE8F8830420BDE8F8830720BDE88F
:10220000F883FFFF2DE9F0470B7807682F2B044672
:102210000E4601D05C2B01D1324601E07B6908E01B
:1022200013782F2B164602F10102F9D05C2BF7D060
:102230000023A36033781F2B04D904F12008DFF8B2
:10224000AC913FE0802384F82B3020460021BDE88C
:10225000F047FFF764BE04F11F00002113F8012FBF
:102260002E2A01F101013CD02F2A3FD1202A0E4411
:102270008CBF2023242384F82B3000212046D4F85F
:1022800000A0FFF74CFE054630B9A1695046FFF7A4
:10229000D1FB0546002873D094F82B30002D40F078
:1022A00087805A0700F19E80A379DB0640F1938076
:1022B00023693878C3F3080307F134011944FFF7A1
:1022C00004FBA0600B2220214046FFF779FA334639
:1022D00013F801292E2ABED000211A4608460825E7
:1022E0002AE003294AD000F8012FB7E75C2ABDD0C5
:1022F000202ABBD942E02F2B25D05C2B23D02E2BBC
:102300006BD08D423AD913F0800F18BF03F07F03D2
:10231000DFF8DCC018BF19F803301CF801EFBEF17C
:10232000000F1AD1A3F1610EBEF1190F01D8203BA5
:10233000DBB208F80130013112F8013F202B00F127
:102340000100D8D80CE0321801E05C2D08D1901BB8
:1023500012F8015B2F2DF8D1F9E77345DDD10DE0BF
:1023600061B194F82020E52A04BF052284F82020DA
:10237000202B8CBF0023042306447CE7062531E094
:10238000E069037893B1C37A03F03F03A371C37A82
:10239000190706D40B224146FFF718FA00283FF42C
:1023A0007BAF00212046FFF7D1FE6CE7042573E7E1
:1023B000042D17D113F0200F03F0040306D0002BD7
:1023C00080D0802384F82B3000250BE0002B14BF35
:1023D0000425052506E0052504E00B2DCED00821B7
:1023E0000B25A9E72846BDE8F08700BF5E7B00000B
:1023F000177B000070B5044605680E460420A169ED
:1024000009B32846FFF716FBF8B9E3691A78FAB161
:10241000DB7AE52A03F03F03A3710DD02E2A0BD0FF
:102420000F2B09D023F02003A3F10802534253419C
:10243000B34201D1002070BD00212046FFF786FE87
:102440000028DCD001E00028F4D00023A36170BD97
:102450000420FAE738B5002104460568FFF75FFD60
:1024600070B9A1692846FFF7E5FA48B9E3691B7816
:10247000E52B08D03BB101212046FFF767FEEFE7CF
:10248000042808BF072038BD70B505460668FFF769
:10249000E1FF044690B9A9693046FFF7CBFA04463C
:1024A00060B901462022E869FFF78AF90B2205F19D
:1024B0002001E869FFF700FA0123F370204670BDA0
:1024C0001FB5019004A8009140F8041D1446FFF7C1
:1024D00097F9002812DB0C4B53F820200AB1002199
:1024E0001170019A0AB10021117043F820203CB10B
:1024F000002201A96846FFF7F1FA02E00B2000E094
:10250000204604B010BD00BFB89002202DE9F04F66
:102510008FB0154601910446002800F0BE8002F0FD
:102520003F073A4602A901A8FFF7D8FA0646002855
:1025300040F0BD800DF13809029B49F82C3D01990E
:102540004846FFF75FFE20B99DF93730002BB8BF32
:10255000062015F01C0F50D040B1042802D1484687
:10256000FFF792FF47F0080748B19DE09DF8123051
:1025700013F0110F40F09780680700F19080390741
:1025800049D50A9DDDF808B029469BF80000FFF701
:102590009CF921234FF0000A2B744C2385F80EA0E0
:1025A00085F80FA06B740A9B2022DA72804652468F
:1025B0000A995846FFF797F90A9B83F81CA083F8FD
:1025C0001DA083F81EA083F81FA0029B0122DA70D1
:1025D000B8F1000F1DD05246414648461D6BFFF72B
:1025E00056FD002860D129460298FFF723FA029B86
:1025F00008F1FF31D96050B156E0002854D19DF860
:102600001230DA064DD4AD0701D5D8074BD43907BF
:1026100001D547F04007DDF808800A9DD8F8303032
:102620002362656298F800002946FFF74EF90146DB
:10263000A06005F11C00FFF7B3F8B8F80630A380DE
:10264000BA064FF000030546E060C4F80080277426
:102650006374E36163612ED568B3B8F80A70606192
:102660007F02AF420CD22068FFF7FFFB0128014632
:10267000A5EB070503D9431CF3D1012600E0022690
:10268000A161A6B9C5F30803ABB10298FFF7ACF896
:1026900060B100EB5520E0610DE009200CE008205E
:1026A00002E0042000E00720064600E002260023A6
:1026B0002360304600E000200FB0BDE8F08F2DE928
:1026C000F74F984600230F46C8F8003001A9064688
:1026D0001446FFF7D9F8002840F08280707C00286B
:1026E0007ED1337CDA077AD5F3687069181A844290
:1026F00028BF0446002C70D07369C3F30802002A77
:1027000048D1019AB2F80A9009F1FF3919EA532920
:1027100010D10BB9B06803E0B1693068FFF7A5FBD1
:10272000012801D8022002E0431C02D1012070746C
:1027300056E0B061DDF804B0B1695846FFF754F8CF
:102740000028EFD0650A09EB000A21D0BBF80A3057
:102750009BF8010009EB05029A4288BFC9EB03050B
:102760002B465246394601F047FA0028DED101993E
:10277000CB785BB1086BCAEB0000854206D94FF4F9
:102780000072343107EB4020FFF796F86D0219E034
:10279000C6F81CA07569F1690198C5F30805C5F56F
:1027A0000075A54228BF2546FFF744F90028BDD192
:1027B000019973693431C3F308032A461944384632
:1027C000FFF77AF8D8F800302B44C8F80030736966
:1027D000641B2F441D4475618CE7204600E00720F0
:1027E00003B0BDE8F08F2DE9F74F9B4600238946E3
:1027F000CBF8003001A904461646FFF745F800283B
:1028000040F0AB80607C002840F0A780237C9A07D2
:1028100040F1A2806369F3424CD3DE434AE063692E
:10282000C3F30802002A7AD1019A5789013F17EAB7
:10283000532742D00198E369026B9A425CD0DDF8DD
:1028400004A0A1695046FEF7CFFF002847D0750AC3
:1028500007EB000855D0BAF80A309AF801007A1947
:102860009A4288BFDD1B2B464246494601F0E1F9FA
:102870000746002837D10198016BC8EB01018D4252
:1028800008D94FF4007209EB41213430FFF714F8F6
:10289000019BDF706D02DBF800302B44CBF8003079
:1028A0006369761BA9441D44E3686561AB422CBF94
:1028B000E360E560002EB2D109E01BB9A06860B901
:1028C000014600E0A1692046FFF76AFB28B9237C96
:1028D00043F04003237400203FE0012801D102208F
:1028E00002E0431C02D10120607436E0A368A061BD
:1028F000002B9FD1A0609DE7FFF72FF800289ED006
:10290000F1E76269E3689A4207D35046FFF725F87A
:102910000028E8D1019BC3F83080C4F81C806569A9
:10292000E1690198C5F30805C5F50075B54228BFF2
:102930003546FFF77FF80028D5D101986369343018
:10294000C3F308032A4618444946FEF7B5FF019B26
:102950004FF00102DA709EE7072003B0BDE8F08F68
:102960000A29F7B504460F4602D10D21FFF7F8FFFB
:102970006368002B14DB5D1C23443B2DA6681F738A
:102980000BDD01AB2A4604F10C012068FFF72BFF99
:10299000019B5D1B18BF4FF0FF3501366560A660D7
:1029A00003B0F0BD4268002A13B5044602DA4FF0C6
:1029B000FF300CE000F10C0101AB0068FFF713FFE2
:1029C0000028F4D16268019B9A42F0D1A06802B05D
:1029D00010BD73B501A90646FEF756FF054648BB74
:1029E000337C5B0626D5316A0198FFF723F805464C
:1029F00000BB746AE37A43F02003E372B268306884
:102A00002146FEF770FFF16804F11C00FEF7D0FECE
:102A1000212323760198A5754C2363760123E57560
:102A2000A574E574C370FEF7BAFF337C23F040034E
:102A300005463374284602B070BD13B50446FFF74F
:102A4000C8FF28B901A92046FEF71EFF00B9206083
:102A500002B010BD07B502AB43F8040D1846FEF7EF
:102A6000CFFE0028A9BF034B0B201870002003B035
:102A70005DF804FBB490022030B58FB000220190C5
:102A800002A901A8FFF72AF8044600BB0EA8029B82
:102A900040F82C3D0199FFF7B5FB044690B99DF92C
:102AA0003730002B03DA029B059A5A610FE09DF83C
:102AB0001230DB060AD5029D0A992878FEF705FF39
:102AC000686104E0042808BF052400E005242046CE
:102AD0000FB030BD2DE9F04395B00022019088463B
:102AE0000270064602A901A8FEF7F8FF0746002873
:102AF00040F09280029B09935B690B934546DDF899
:102B00002C90B9F1000F5BD0202109A8FFF707FA3C
:102B10000446002852D10F990298FEF78BFF044615
:102B200000284BD1029B10991878FEF7CEFE214663
:102B30000B9009A8FFF7F3F9044600283ED10021C5
:102B400009A8FFF757FC0446002861D1029B1099A1
:102B50001878FEF7BAFE814508D10F9B8DF8154015
:102B600093B103A909A8FEF7CAFE07E0214609A808
:102B7000FFF7ECFA04460028E1D049E003AB234418
:102B80005B7A13B10134F9E71C46631C9D4214D3F0
:102B9000281B2B46C5EB040E8342019908D0013B4C
:102BA00003EB0E020DF10C0C6244527ACA54F3E7A7
:102BB000E44325442F234B55A1E7112427462BE05E
:102BC000454503D1013D019B2F225A55154B1A78DB
:102BD000154B53F822201146881A11F8013B002B9F
:102BE000FAD1811C8D4211D3834203D0D15CF154C0
:102BF0000133F9E733443A225E1C1A70019B5B5D96
:102C000006F8013B0135A845F8D805E0112703E097
:102C1000042C08BF0224D1E700233846337015B0D6
:102C2000BDE8F083B4900220EC7B000073B50D4644
:102C300001A90446FEF728FE002876D1607C002812
:102C400073D1E368AB4204D2227C12F0020F08BFBA
:102C50001D46002263696261002D64D0019A568985
:102C600076026BB1013B6A1EB3FBF6F1B2FBF6F2E2
:102C70008A4205D3724213406361ED1AA16910E0E4
:102C8000A16869B92046FFF78BF90128014601D1F7
:102C9000022002E0013002D10120607445E0A16011
:102CA000A161B9B900232CE0636933446361237CDB
:102CB0009A07A5EB060510D52046FFF771F90146E6
:102CC00080B14B1CE8D00129E2D9019B9B69994254
:102CD000DED2A161B542E7D805E02068FFF7C5F86C
:102CE0000146EEE7054663692B446361C5F30803BB
:102CF000002BD7D00198FEF777FD0028C8D000EB55
:102D00005523E2686569954281BF227CE56042F007
:102D100040022274C5F3080038B1E2699A4218BF34
:102D2000E361002001E02B46F4E702B070BD1FB55F
:102D30000446019138B3002203A901A8FEF7CEFE94
:102D4000F0B9039B236001992046FFF75BFA00BBB3
:102D500094F92B30002B08DBA379DB060FD5039BFE
:102D6000E1691878FEF7B1FDA060039BDB88A380C2
:102D700000212046FFF7D3F80428034605D105209B
:102D80000023236008E0092006E0002BF8D1184654
:102D900002E00428F3D0F3E704B010BD13B501A995
:102DA0000446FEF771FD00B9206002B010BD37B5D2
:102DB0000D4601A90446FEF767FDC0B9014620464D
:102DC00015B9FFF7ACF812E0FFF714FB10F0FB03A6
:102DD0000DD16B72A3691BB129462046FEF78FFD0A
:102DE00000212046FFF7B2F9042808BF002003B0F5
:102DF00030BD30B58FB00D460190002203A901A867
:102E0000FEF76CFE044698B9019903A8FFF7FAF99A
:102E1000044668B99DF93730002B08DB45B1099BA2
:102E200068722BB1294603A8FEF769FD00E006246D
:102E300020460FB030BD2DE9F04385B088460190A3
:102E4000154603A9002201A8FEF748FE0646002801
:102E500051D1039C2C60A7692369BA1E934202D802
:102E6000C8F8003047E02378012B11D1022705462E
:102E700039462046FEF7F9FF431C2FD001282FD0FA
:102E800000B90135039B9B6901379F42F0D32AE0CB
:102E9000616A0546044634B9039801F10109FEF759
:102EA000C9FDF8B94946039810F8343B022B08D104
:102EB00003195A78035D53EA022308BF013502342F
:102EC00007E02044FEF76CFC20F0704000B90135AB
:102ED0000434013FC4F30804DDD104E0012602E01C
:102EE000022600E00646039BC8F800501A791D61CF
:102EF00042F001021A71304605B0BDE8F08373B5A7
:102F000001A90546FEF7C0FC002833D16C7C84BBC8
:102F10002B7C9A072BD56E69EB689E4229D23EB96D
:102F20002246A9682846FFF7B2F8AE60044615E0CD
:102F3000A9692868FEF799FF431C014603D00128C0
:102F400003D102240AE0012408E0019B9B69984216
:102F500004D2AA692846FFF79AF804466B69EB6029
:102F60002B7C43F040032B741CB16C7401E00720F0
:102F700000E0204602B070BD2DE9F0419AB0022277
:102F8000019003A901A8FEF7A9FD0446002851D12C
:102F90001AAE039B46F8583D01993046FFF732F9C7
:102FA0000446002846D19DF83B309A0607D41B06FC
:102FB00005D49DF8168018F0010F1FD101E00624FA
:102FC00038E0039F0B993878FEF77FFC18F0100F5C
:102FD000054615D07B699D4210D021460FA80F975A
:102FE0001195FEF79CFF044620BB01460FA8FFF792
:102FF00001FA044610B1042802D01BE0072419E0AE
:10300000049F0A993846FEF715FD044690B90B9BBC
:10301000E5221A700123FB7025B90398FEF7BFFC67
:10302000044607E0224629463046FFF730F80446BA
:103030000028F2D020461AB0BDE8F0812DE9F04F0B
:1030400093B00222019002A901A8FEF747FD0446B1
:10305000002840F0868012AE029B46F82C3D019974
:103060003046FFF7CFF80446D0B1042879D19DF857
:10307000473003F0200303F0FF019BB912AF029B1E
:1030800047F83C3D3846FEF78BFF054660B1012D01
:103090000CD10224002229463846FEF7F8FF60E0F2
:1030A00008245EE006245CE00724F3E76B1C56D09E
:1030B00029460298FFF721F804460028EAD1029831
:1030C0000B2220213430FEF77BFB02984FF02E08B4
:1030D0004FF010094FF0210B4FF04C0A80F834806C
:1030E00080F84A4080F84B4000F1340180F83F906E
:1030F00080F84CB080F84DA02A46FEF7F4FB029809
:10310000202200F134015430FEF7D6FB0298099AD0
:1031100080F8558000F15401FEF7E5FB029B4FF06B
:10312000010883F803803046FFF7AEF90446002813
:10313000B0D10E9B9875D87583F818B083F819A094
:103140002A460E990298FEF7CEFB0E9B029883F852
:103150000B9080F80380FEF722FC044601E0012476
:1031600098E7204613B0BDE8F08F70B5A2B001908B
:1031700022A840F8881DFEF743FB022203A901A8FC
:10318000FEF7ACFC002875D122AC039B44F8583DF7
:1031900001992046FFF736F800286BD19DF85B3087
:1031A00013F0A00F52D12022139904A8FEF784FB3C
:1031B000214617A82C22FEF77FFB009917A8FFF7DE
:1031C00021F840B90E9B199A9A4250D1109B1B9A34
:1031D0009A424CD101E004284CD117A8FFF754F9CA
:1031E000002847D11E9C13220DF11D0104F10D0092
:1031F000FEF762FB9DF81B30039DDA0658BF43F0D3
:1032000020030126E372EE70E37ADB0620D5199BDA
:103210000E9A9A421CD021462878FEF756FB0146AA
:103220002846FEF7E1FA014618B32846FEF702FCED
:1032300000BB039890F855302E2B09D1199A00F154
:103240005401FEF750FB039BDE7001E0062011E005
:103250000C9C12992046FEF7EDFB58B9139BE52212
:103260001A700123E3700398FEF799FB02E008202F
:1032700000E0022022B070BD30B58FB00C46019046
:10328000154602A9022201A8FEF728FCE8B90EA8FB
:10329000029B40F82C3D0199FEF7B4FFA8B99DF8B8
:1032A000373013F0A00F0FD10A9A0298D17A84EA2E
:1032B000010305EA030404F027044C400123D472FF
:1032C000C370FEF76CFB00E006200FB030BD10B5F8
:1032D0008EB00C460190022202A901A8FEF7FEFB67
:1032E000D8B90EA8029B40F82C3D0199FEF78AFF41
:1032F00098B99DF8373013F0A00F0DD1E388A1885D
:103300000A9843EA01411630FEF752FA0298012367
:10331000C370FEF744FB00E006200EB010BD70B590
:103320008EB00D460190164602A9002201A8FEF7B4
:10333000D5FB044600283FD135B3029B05900146DA
:1033400003A80393FEF7EBFDD0B9012103A8FFF713
:1033500051F8A8B90A9B6A1E013B05F10A0113F84E
:10336000010F02F8010F9142F9D105F10B03002181
:103370009D42197008D013F8012D202AF8D003E0DF
:10338000042818D100232B70B6B10298016AFEF709
:1033900051FB044680B9029B1A78032A04D0042A00
:1033A0000CBF6420272000E0432034331844FEF78C
:1033B000F7F9306000E0044620460EB070BDFFFF14
:1033C00030B595B00222019002A901A8FEF786FB54
:1033D000044600285CD103AD28460B222021FEF7CD
:1033E000EFF93048019B1A781F2A1AD95A1C01920A
:1033F0001A7893B2A3F16101192902D8203B9BB23C
:1034000007E07F2B84BF121812F8803C0BB906200E
:1034100045E0254911F8012F002A3BD09342F9D10C
:10342000F5E79DF80C30E52BF1D02CB1631EEA5C7A
:10343000202A01D11C46F8E7029B0993002109A824
:103440000B91FEF76CFD50BB012109A8FEF7D2FFDE
:1034500020B994B9109BE5221A7013E004281ED1FC
:10346000B4B109A8FEF7F6FFC8B9202201461098AA
:10347000FEF7A6F9109B0822DA720B222946109853
:10348000FEF71AFA02980123C370FEF788FA06E0E5
:10349000204604E00B2CBAD02B550134A2E715B01E
:1034A00030BD00BF5E7B0000FB7A00002DE9F74FC6
:1034B0000E4601A904461746FEF7E6F9002879D121
:1034C000607C002876D1002E5BD0E368002B58D1B9
:1034D000237C9A0755D5019A5389D2F80C805B0258
:1034E000B6FBF3F5013B3340002B18BF0135B8F1B3
:1034F000010F05D99369984528BF4FF0020801E0F4
:103500004FF00208C146C2464FF0000B51462068FA
:10351000FEF7ABFC019B9B690AF1010A9A4528BFA3
:103520004FF0020A012828D0431C28D020B90BF103
:10353000010B5D4503D105E0D1464FF0000BC245BC
:10354000E4D11EE017B909F1FF301CE0C846AA46D5
:10355000BAF1000F17D0BAF1010F14BF08F1010240
:103560004FF0FF3201984146FEF704FC10BB404685
:103570000AF1FF3A08F10108EAE702201AE0012007
:1035800018E0072016E0019BD86097B1227CC4F8B0
:10359000089042F04002227499691A69E660023983
:1035A0008A429FBF551B1A791D6142F0010298BFE4
:1035B0001A71002003B0BDE8F08FFFFF2DE9F04F36
:1035C0008DB00DF1300E0D464EF80C0D70461746BD
:1035D0001C46169EFEF714F90028C0F29382B74BE2
:1035E00053F820300BB100221A705FFA80FA0121E3
:1035F000504600F0EDFAC20700F18682430700F161
:1036000085820AAA0321504600F030FB30B90A9A9D
:10361000531EB3F5004F01D21A4201D001230A9381
:1036200037B1A74BA7F500729A4201D9132081E266
:103630007B1E3B42FAD1002C00F06A82730A03938E
:1036400000F066820BAA0121504600F00FFB002813
:1036500040F0608205F0080303F0FF02002B0CBF6E
:103660004FF03F094FF000090B9B0292994501D999
:103670000E205FE2C9EB03037F2B0B93F8D97A0A84
:10368000802AD3D805F0020101F0FF00049029B18F
:1036900005F00701022905D0E80703D5E907C5D5DC
:1036A000022700E00327190B06910A99481E494298
:1036B0000791032F4FEA53410890059140F6F57C9E
:1036C0004FF6F57E72D14AB97E48012630F8021FC6
:1036D00029B1059D8D4202D37600F7E71646B3FB6C
:1036E000F6F179488D00A1F57F41F63905F20725FD
:1036F00081424FEA5525BBD8002101914FF0200BA4
:103700001EE0069D8D4204D3760030F8021F00298A
:10371000F7D1B3FBF6F565459BBF05EB45050135D4
:1037200002356D088CBF6D00033505F2FF154FF0B3
:1037300020018CBF022701276D0A01914FF0010B78
:103740000BEB0901009101990098691801EB000841
:1037500008980799032F404400EA010008BF009928
:10376000C8EB000006BF091883442D18C9EB0610EA
:1037700008BF009108EB00018B42FFF479AFCBEB5F
:1037800003080199C5EB0808032FC1EB0808B8FB33
:10379000F6F811D0022F22D1F04516D9002A40F0B8
:1037A000C3817600402E00F2B781324612B94748F5
:1037B0000126AAE71646ACE7F04516D8002A7FF4A2
:1037C00057AF72083FF454AF7DE7E0450DD8002AAB
:1037D0007FF44EAF7200802A3FF64AAFE6E740F62C
:1037E000F57398453FF644AF01274FF4007200216E
:1037F0002046FDF7E5FF0B2235492046FEF75CF831
:103800000B9984F80EB000230222032FE372227377
:10381000CBF3072B4FF00102637418BF0223B1F5FD
:10382000803F667384F80FB02274A37404D2E174ED
:10383000C1F30721217503E004F12000FDF7B8FF73
:10384000F82363753F2300222376FF23A376627655
:10385000E276494604F11C00FDF7AAFF032F4FF062
:10386000210339D184F845304C2384F8432084F86F
:10387000442084F84630294604F12400FDF798FFDF
:10388000022384F82C30012384F83030062384F896
:103890003230802384F84030292384F82D2084F8A6
:1038A0002E2084F82F2084F8312084F8332084F8E7
:1038B00042301322074904F1470024E0B890022067
:1038C00000FEFF00DC7B0000FFFFFE0FEC7A000033
:1038D000277B0000337B000084F829304C2384F8D8
:1038E0002A30C5F30723E375802384F824309349F5
:1038F00084F82720292384F82820A57584F8263009
:10390000132204F12B00FDF7D7FF4FF0550384F885
:10391000FE316FF0550384F8FF314A4601232146FA
:10392000504600F086F98346002840F0F380032FCC
:1039300041D1012309F106022146504600F079F9F0
:103940004FF4007259462046FDF73AFF52234122B8
:103950007221237063706123A370E27084F8E41114
:1039600084F8E51184F8E62184F8E73108F1FF31A5
:1039700004F5F470FDF71CFF022384F8EC314FF0DE
:10398000550384F8FE316FF0550384F8FF3109F1D7
:1039900007020123214684F8EDB184F8EEB184F8E2
:1039A000EFB1504600F045F9012309EB030221462F
:1039B000504600F03EF9039B00215A022046FDF7D5
:1039C000FFFE032F0FD1F8232370FF236370A37032
:1039D000E37023716371A371E37123726372A37245
:1039E0000F23E37207E0012F5549204618BF6FF0FF
:1039F0000701FDF7DDFE039B009AAB4228BF2B4673
:103A000021465046984600F014F90146002840F03F
:103A100081804FF400722046FDF7D2FE009BB5EB8B
:103A2000080543440093E6D1019B032F08BF3346AA
:103A30000193019B039A934228BF13462146009AA3
:103A400050461D4600F0F5F8002863D1009B2B443A
:103A50000093019B5B1B0193EBD1032F08D00B9BC1
:103A6000B3F5803F06D2022F14BF0123042302E0E6
:103A70000C2300E00623029A42B100221146504670
:103A800000F0F4F8003018BF012053E04FF400724A
:103A900002992046FDF794FE552284F8FE21AA22C1
:103AA00084F8FF219DF8082084F8BE2184F8C12104
:103AB0000B9A84F8C2314A4443F6C163B2FBF3F275
:103AC000FE2384F8C331930843F03F03012584F8B3
:103AD000C43184F8C521494604F5E37084F8BF5128
:103AE00084F8C051FDF764FE0B9904F5E570FDF70D
:103AF0005FFE2B46029A2146504600F09AF80028B5
:103B0000BBD007E00B2015E0032013E00A2011E0F2
:103B100011200FE001200DE0049909B10327D3E53E
:103B2000802E3FF6A5AD40E6049900293FF4A0ADF4
:103B30000327C8E50DB0BDE8F08F00BF477B00004C
:103B4000F8FFFF002DE9F341064690464F1E04465C
:103B50000025BD4213DA01AB012269464046FEF75B
:103B6000AEFD019B012B0AD19DF800300D2BF0D04A
:103B7000621C0A2B237005F101051446E9D10023CC
:103B80009D4214BF30461846237002B0BDE8F08154
:103B900010B594B003464C220C4601A80021FDF755
:103BA0000FFE01A819460194FEF7DAFE01A8FEF700
:103BB000F9FE14B010BDFFFF012803D820B9034B54
:103BC0001878704701207047032070474087022013
:103BD00010B558B902F072FC044602F069FB044BC0
:103BE0001870044B04B91C70187810BD032010BD68
:103BF000C89002204087022070B504460E46194640
:103C0000FFF7DAFFC3070ED46CB961B114468D1803
:103C10002146304602F05EFB06F50076013420B9FD
:103C2000AC42F5D101E0032070BD003018BF012087
:103C300070BD70B504460E461946FFF7BDFFC307B9
:103C40000ED46CB961B114468D182146304602F08D
:103C5000C3FB06F50076013420B9AC42F5D101E092
:103C6000032070BD003018BF012070BD10B50446A0
:103C7000FFF7A2FFC3070DD464B9012904D00BD309
:103C8000032904D0042010BD4FF0807300E080238E
:103C9000136001E0032010BD204610BDFCF792BF69
:103CA0002DE9F0478046006818B3064601303378A6
:103CB000202BFAD0DFF8409000252C0154F809A001
:103CC000504603F01DFA314607460246504603F0BF
:103CD00085FA48B94C442379012B05D13E44C8F8F4
:103CE00000606079BDE8F08701351A2DE5D14FF00D
:103CF000FF30BDE8F08700BF38800000132833D8BC
:103D0000DFE800F0300A0C0E10121416181A1C1EF0
:103D100020222426282A2C2E154826E0154824E0A7
:103D2000154822E0154820E015481EE015481CE023
:103D300015481AE0154818E0154816E0154814E033
:103D4000154812E0154810E015480EE015480CE043
:103D500015480AE0154808E0154806E0154804E053
:103D6000154802E0154800E01548FCF753BF00BFB6
:103D7000FC7B0000087C0000197C00002A7C00000D
:103D80003A7C00004A7C00005D7C00006D7C0000F5
:103D9000837C0000997C0000B17C0000CB7C00009B
:103DA000DE7C0000077D0000187D0000377D0000EC
:103DB000487D00005E7D0000747D00008B7D00006A
:103DC000957D0000B1F57A7F4FF47A7335BF434398
:103DD000B1FBF3F1B3FBF1F3B0FBF1F301460148A2
:103DE000FDF710B8A57D00002DE9F0410E468EB01C
:103DF0001446014678B3B6F5806F2CD3012204A88F
:103E0000FEF784FB054698B9174B1B680293DDF853
:103E10000880074601AB4FF40072314604A8FEF754
:103E20004EFC054638B9019B2BB11F441E44F1E7F7
:103E30004FF00008474604A8FEF7FFFD6DB974B1C6
:103E4000094B0A4A1B68039303993846C1EB0801E2
:103E5000FFF7B8FF01E0132002E0284600E020460B
:103E60000EB0BDE8F08100BFC09C0220C67D0000FE
:103E70002DE9F047144608AE00221D4696E8C0031F
:103E8000FFF7B2FF70B9013425B1012D0AD144F01A
:103E9000010420474B46424639463046A446BDE819
:103EA000F04760474FF0FF30BDE8F0872DE9F0475D
:103EB0009DF82090074690469A4646180446C7EB60
:103EC0000A0121443448FCF79DFF3448FCF7A2FE68
:103ED00000254D452FD2B8F1100F04EB050303D098
:103EE000B8F1200F0CD017E09E4204D919882C4855
:103EF000FCF788FF02E02B48FCF78CFE023516E049
:103F00009E4204D919682448FCF77CFF02E0264849
:103F1000FCF780FE04350AE09E4204D91978234854
:103F2000FCF770FF02E02248FCF774FE0135202008
:103F3000FCF74AFECDE71F48FCF76CFE04EB0905D1
:103F4000A5420BD0A64204D92078A0F120035E2B15
:103F500000D92020FCF738FE0134F1E71648FCF7C1
:103F600059FE01F0BBFE40B220280DD101F0B6FE93
:103F700040B2202803D1AE4209D92C469FE71B2826
:103F8000F4D10020BDE8F0871B28F4D1F9E74FF009
:103F9000FF30BDE8F08700BF757700007A7700003A
:103FA000CB7D0000D47D0000D07D00007E77000036
:103FB000D67D0000837700008677000010B50949A0
:103FC00004460948FCF71EFFFCF7F4FD074A0849C0
:103FD0000848FCF717FF1CB1BDE81040FCF74CBDCA
:103FE00010BD00BFD97D0000DD7D0000E67D000032
:103FF000F17D0000F77D000070B5174C0A460D46B4
:104000000021064602F09CFF23784BB90122134998
:104010001348FEF77BFA08B1022300E00123237066
:104020002378012B0ED10E4A29463046FFF78AFD30
:1040300010B1FCF7EFFD05E00948FEF7FEFC064B6A
:1040400002221A702378022B04D1064A29463046F0
:10405000FDF71EF9002070BDC9900220087E000007
:10406000CC900220157E00002DE9F043974EA9B0B8
:1040700000200121C6F84C0BFFF7AAFD0AAC05464B
:1040800020B19348FCF7BEFE00270CE09149204682
:10409000FCF7C6FE2A46214606F17C00FEF710FA20
:1040A0000028EED101278C48FCF7B4FD782120468A
:1040B0000494FFF7A1FF04A8FFF7F2FD422800F0E7
:1040C00044810FDC3D285BD004DC0028EBD03C2889
:1040D0001ED0DAE1402800F0848000F3DE803F2823
:1040E00033D0D2E1792800F0B38106DC432800F018
:1040F0006681782800F09D81C7E1832800F0BD81AA
:10410000852800F0BF81822840F0BF817348C1E05C
:1041100005A904A8FCF7EAFE0028C4D006A904A853
:10412000FCF7E4FE0028BED007A904A8FCF7DEFED9
:1041300000B907906A48FCF76DFD059B069A9A4204
:104140001CD9079A43F8042BF8E705A904A8FCF743
:10415000CDFE0028A7D006A904A8FCF7C7FE0028BA
:10416000A1D007A904A8FCF7C1FE00289BD05D4898
:10417000FCF750FD0599069B8B4222D85A4889E0EE
:1041800005A904A8FCF7B2FE00288CD006A904A853
:10419000FCF7ACFE002886D007A904A8FCF7A6FE11
:1041A000002880D05148FCF735FD059A069B9A42BD
:1041B000E4D2079B12F8011B1970079B0133079388
:1041C000F4E7079B0D46187815F8012B904203D0B1
:1041D00000904748FCF716FE079B013307932946DA
:1041E000C9E705A904A8FCF781FEC0B9414B93F8C3
:1041F00034200AB19B6911E093F835200AB11B689D
:104200000CE093F836200AB19B6807E093F837205A
:104210000AB11B6902E09B6AA3F50073059306A926
:1042200004A8FCF763FEB8B9324B93F834200AB106
:10423000DB6910E093F835200AB15B680BE093F876
:1042400036200AB1DB6806E093F837200AB15B69D3
:1042500001E09B6A0833069307A904A8FCF746FE11
:10426000002800F05F81079B083B182B00F25A8161
:10427000214A22FA03F3DB0740F154811F48FCF77F
:10428000C9FC20230093059B079A06991846FFF75F
:104290000DFE1B48FCF7BEFC05E705A904A8FCF7CA
:1042A00025FE00283FF4FFAE06A904A8FCF71EFE79
:1042B00068B3059B5A1C0592069A1A7006A904A8B1
:1042C000FCF714FE0028F4D1EDE600BFF4900220C4
:1042D0001D7E0000547E0000577E0000267F0000F7
:1042E0005A7E0000727E0000067E0000677E00009D
:1042F0007F7E00000087022001010001997E0000FE
:10430000A67E00001F2B11D8059B0133059305994C
:1043100086480A78FCF776FD78212046FCF7AAFD4E
:104320009DF8283004942E2BECD1BCE606A904A8F5
:10433000FCF7DCFD28B1059B5A1C0592069A1A7001
:10434000E5E77B48FCF766FCE1E708A904A8FCF771
:1043500020FE00283FF4A7AE09A904A8FCF719FE27
:1043600080B1089B099A23F8022B09A904A8089395
:10437000FCF70FFE0028F4D195E61F2B11D8089BFF
:104380000233089308996B480A88FCF73BFD7821B3
:104390002046FCF76FFD9DF8283004942E2BECD1BD
:1043A00081E609A904A8FCF7F4FD20B1089B099A4D
:1043B00023F8022BE5E75E48FCF72CFCE2E708A9AE
:1043C00004A8FCF7E6FD00283FF46DAE09A904A897
:1043D000FCF7DFFD88B1089B099A1A60089B09A9C0
:1043E000043304A80893FCF7D4FD0028F3D15AE65F
:1043F0001F2B11D8089B0433089308994E480A686C
:10440000FCF700FD78212046FCF734FD9DF82830AC
:1044100004942E2BECD146E609A904A8FCF7B9FDBB
:1044200018B1089B099A1A60E4E74148FCF7F2FBCF
:10443000E3E705A904A8FCF759FD00283FF433AED3
:1044400005993E48FCF7DEFC059B43F0010318E0AC
:1044500005A904A8FCF74AFD00283FF424AE0599FD
:104460003748FCF7CFFC059B9847014600283FF4EE
:104470001AAE3448FCF7C6FC15E63348FCF7CAFB15
:1044800001231847FCF7F8FA0DE69DF8283004944C
:10449000002B3FF408AE002F40D004A8FCF71BFA15
:1044A000012580464FF00009022D0ED0032D11D0BA
:1044B000012D18D1254B0193CDF80080244B2549BF
:1044C000002214A8FCF7ACFC13E0234914A8FCF765
:1044D000A7FC0EE0CDF800801D4B2049002214A857
:1044E000FCF79EFC05E0434600221D4914A8FCF79A
:1044F00097FC1C4B1C4A0393049B00930296CDF837
:1045000004900023114614A8FFF7B2FC01307FF499
:10451000CAAD042D02D00135EDB2C5E71348FCF752
:1045200071FCC0E508230793A8E600BFB27E000037
:10453000BD7E0000C27E0000CD7E0000D87E00005F
:10454000F37E00000C7F0000417F0000657F0000CB
:10455000547F0000587F0000627F0000697F0000E8
:10456000737F0000008702200000FF1F7A7F000099
:1045700008B5114B00224FF4FA601A700F4AC3F8C5
:10458000502B00F00FF90E4B0E4A1A600E4B0F4ADB
:104590001A60FCF723FAFCF714FB0D48FCF73AFB12
:1045A0000C48FCF737FB0C48FCF70AFB0120FFF72F
:1045B00005FDFFF759FD00BFF4900220C09C0220CA
:1045C000A4A00220255E0000A0A00220DD5C000067
:1045D000887F0000947F00009D3C0000054B187808
:1045E000054B1A78C0B2D3B2984238BF4030C01AD7
:1045F000704700BFB69C02204D9C022010B5284B8E
:104600001A79920620D52749DA790B7826480133A2
:1046100000783F2BC8BF0023834218BF2348D2B283
:104620001EBFC254DAB20A70214A116861B1214A30
:104630001278D2B2934236BFC2F140029B1A9B1845
:10464000272BC4BF01230B701549CA78D2B21406B8
:1046500016D50B79180613D5174B164C18782378F6
:10466000DBB2984202D16C23CB7009E00133282BD6
:1046700028BF00231148C05CDBB2C0B2C8712370F0
:1046800051060CD5064B1A79520608D50C4A002162
:1046900011700C4A126802B111702C22DA7010BD30
:1046A00000C00640B69C02204D9C0220769C022051
:1046B000489C0220B79C0220BC9C02204E9C0220F9
:1046C0004C9C0220B89C022010B572B60B480268C0
:1046D000B2FA82F10B2902DD62B6002010BD4FF064
:1046E0000043CB4022EA0302026062B6044C482336
:1046F0004B43E0180022E250426010BD4487022084
:10470000988302200C4B4822C31AB3FBF2F30B2B05
:1047100011D80A4A127822B1094A12780AB100F077
:104720004FBA72B607494FF0004222FA03F30A6803
:104730001A430A6062B6704798830220A19E022045
:10474000AC9E022044870220044B054900221A60D7
:104750000A60044A106010221A60704714D00340A7
:1047600004D0034000D0034072B60B4B0B4A0C49F7
:104770001B681268096862B6490102D5322B88BFEE
:104780000132C3F53B4330207F33B3FBF0F34FF4EA
:104790007A7000FB0230704718E000E0C09C0220F5
:1047A00004ED00E038B50446FFF7DEFF054624B906
:1047B00038BD013C0AD005F57A75FFF7D5FF401BDF
:1047C000B0F57A7FF5D201F02DFCF6E738BDFFFF9A
:1047D0002B4B4FF0006270B51A604FF080521A6098
:1047E0004FF000521A604FF080421A604FF00042C2
:1047F0001A60244B244A254D254C264E4BF6FF715A
:10480000002018605960282313609360136193613E
:104810001362936213639363103202F501222B60DB
:1048200023601360936013619361136293620922A2
:10483000326006F58056043630607160B3603361D3
:1048400046F8042C06F5FE2630607160B3603361D3
:1048500046F8042C06F5805630600F4801602B6046
:1048600023600E4B1A6001F067F91920FFF79AFFD9
:1048700000F0E4FF40F21310BDE87040FFF792BF74
:1048800004E100E0048003400C8003400C900B40E6
:1048900014900B400080034008900B4000900B40A8
:1048A00030B503460020B3FBF2F402FB1433092BAE
:1048B00094BF30333733DBB20B5423460CB1013095
:1048C000F1E70A1823465470C41AA34206DACC5CF6
:1048D0001578CD5402F801490133F5E7084630BD9B
:1048E000054B1878054B1A78C0B2D3B2984238BF3E
:1048F0004030C01A704700BF329D0220C99C022080
:1049000010B5284B1A79920620D52749DA790B7809
:104910002648013300783F2BC8BF0023834218BFCD
:104920002348D2B21EBFC254DAB20A70214A1168BB
:1049300061B1214A1278D2B2934236BFC2F140022D
:104940009B1A9B18272BC4BF01230B701549CA78EB
:10495000D2B2140616D50B79180613D5174B164C80
:1049600018782378DBB2984202D16C23CB7009E02F
:104970000133282B28BF00231148C05CDBB2C0B232
:10498000C871237051060CD5064B1A79520608D50A
:104990000C4A002111700C4A126802B111702C22CD
:1049A000DA7010BD00B00E40329D0220C99C02207A
:1049B000F29C0220C49C0220339D0220389D0220DC
:1049C000CA9C0220C89C0220349D02201FB572B6EA
:1049D000134B144970221A70134A116080221A7006
:1049E0001A781206FCD5114B186862B6104B984223
:1049F00098BF0A2301AC98BF58430A222146FFF70B
:104A00004FFF0C4A0023E15C21B101330A2B22F84D
:104A1000021BF8D1084A01335B00137004B010BDCB
:104A20000000024000000741040002400C00024068
:104A30007F969800D2870220D0870220054B1878F5
:104A4000054B1A78C0B2D3B2984238BF4030C01A72
:104A5000704700BFC29D0220419D0220F0B534493D
:104A60000B7913F0300F2FD072B68B7D03F0FF045B
:104A700023B9CB7940234B7462B625E062B62D484A
:104A80002D4A037812782D4FDBB2D2B20546581C5E
:104A90004028CE7928BF00209042F6B21CBF3E5479
:104AA0000346601E10F0FF04F1D1D9B229702449E9
:104AB000096849B1934236BFC2F140029B1A9B1864
:104AC000272BC4BF01230B70194AD178C9B20D0638
:104AD0001ED513791C061BD51A4B1B481D7803786D
:104AE0001A4EEDB2DBB2AB420AD00133402B28BFE5
:104AF00000231479F45CE4B2D471147D072CF2D94C
:104B0000DBB203700A4B1A79100644BF7C22DA70BC
:104B100049060CD5064B1A79520608D50C4A0021D5
:104B200011700C4A126802B111703C22DA70F0BDAB
:104B300000A00640C29D0220419D0220829D0220CD
:104B40003C9D0220C89D0220C39D0220429D022060
:104B5000409D0220C49D0220431E032B14D872B630
:104B60000A4951F8230068B170B4094C058834F83B
:104B70001320466841F82360521B24F8132062B6C4
:104B800070BC704762B6704700207047249E0220B8
:104B9000A8A00220013803280BD872B6074B53F89F
:104BA000203043B100205B680130002BFBD162B69E
:104BB0007047002070471846F9E700BF789E022032
:104BC00030B472B62B4A13781D0706D52A4B196AE2
:104BD000002936D0996A002941D053781C0706D5A0
:104BE000254B196C00293ED0996C002939D0937857
:104BF000190705D5204B196E002936D0996E89B159
:104C0000D3781B0707D51C4BD3F880207AB3D3F891
:104C1000882011213AB162B6184B00221A7030BCBC
:104C2000FFF770BD0D21154C154D227843F831501A
:104C300003EBC1030830013A5860227062B630BC01
:104C4000704704220D4C0F4D217843F8325003EB8E
:104C5000C20308304A1E5860227062B6EFE7052191
:104C6000E1E70921DFE70822ECE70C22EAE710225E
:104C7000E8E700BFD881000000800220A19E02204A
:104C8000C800400088004000431E032B1DD81B4A6B
:104C9000400140F0100030B4104472B6184CE25C91
:104CA000032A1BD8DFE802F00212151703220D8831
:104CB000E25410F0080F14BFC823882343EA0543C9
:104CC00008310360416062B630BC70470830022290
:104CD000EDE70522EBE708300422E8E7094A52F83D
:104CE000230038B1084A52F82300416042F82310EB
:104CF00062B6E9E742F82310034AF7E70080022092
:104D0000B09E0220789E0220889E02202DE9F04F5E
:104D1000B54CB64E87B046E0B54F4FEA930B07EB64
:104D2000CB08013DD8F8041003F00803EDB2A1F15F
:104D3000080003F0FF02002B40F0108157F83B30D1
:104D40001B0C1FFA83FE21F808EC002B00F0FD80FD
:104D5000A84B21F8062C41F8042C53F82520002AF2
:104D600000F0DF82DFF8CCA25AF825305860DFF877
:104D7000C8924AF8250039F815309E4429F815E004
:104D8000FFF7A2FC002800F0C5829B499B4B18F05E
:104D9000080F00F1080018BF0B46C8F8040047F8D8
:104DA0003B30082323702578EDB2690719D5944B61
:104DB0001B78A3B193490A7802F0FF0322B1013BAB
:104DC000DBB20B7003B900BE8F490A7802F0FF0313
:104DD0002AB1013BDBB20B70002B00F0718204237F
:104DE000237005F0080303F0FF02002B00F0DC80C5
:104DF0003378DBB21D098FD19B087D4D55F83320E8
:104E000005EBC301C2F38302013A49680C2A00F2A0
:104E10009880DFE802F08C8C9696969696964D9642
:104E2000969607000868DFF8F4E14A68DFF80CB2EC
:104E3000764FCEF80420CEF8000082B240F28160B6
:104E40000021DFF8B49145F833904FF0010C824215
:104E5000CBF800102961A96187F800C0DFF89091B4
:104E600000F2F080B2F5D06F80F08F83B2F5817FD1
:104E700000F0218300F2A882802A00F06283822A57
:104E800040F02083BEF8043003F07F03042B00F2CF
:104E900019835F4A5F489B001A4401704170137880
:104EA0009B0740F17A8480F800C04FF0020C4DE37C
:104EB000DFF888B1DBF8003073B3DFF884A1534F1B
:104EC000554ABAF8001097F800E0107840298C464F
:104ED00040F0020928BF4FF0400CBEF1000F8EF0E9
:104EE000010E87F800E0CCEB01010CBF8827C82732
:104EF00005EBC90E89B280F0010047EA0C47CEF8F5
:104F00000430AAF8001045F8397063441070002985
:104F100000F04581CBF80030404B1A88B2F5A06F05
:104F20000FD13F4A9978117000225A7009E03B4A2C
:104F3000108842F22102904200F036812E4A45F854
:104F40003320384A012313702BE72B492B4B18F0E1
:104F5000080F18BF0B4647F83B3022E7FFF7D2FB9C
:104F60003148324A50F82510002900F013824B686E
:104F700012F805C040F8253001F10803C8F80430E4
:104F8000BCF1030F05D8DFE80CF02C022926022320
:104F9000535518F0080F0A880CBF8823C82343EA2A
:104FA000024347F83B30FCE6E80700F18C81290614
:104FB00000F10082AA0706D51D4A0B49137802208A
:104FC000DBB213700870EB0602D5074B10221A7083
:104FD00007B0BDE8F08F04235355DAE70523535596
:104FE000D7E703235355D4E780200740902007409C
:104FF00000800220249E0220C8004000880040005B
:10500000AC9E0220359E022019A00220349E022070
:10501000C0200740A49E0220A09E0220989E02204D
:105020009820074094200740789E0220B09E0220DE
:1050300088200740D09D0220A8A00220CC9D0220FD
:10504000E09D022042F221039A4200F0358100F2F5
:10505000D980B2F5086F00F0B382B2F5106F40F05E
:105060003182B24AD9F820309EF8021011701A0627
:1050700000F14383AB6AAE4A1B0600F139832B6B08
:10508000AB4A180600F14E83AB6BA94A190600F132
:1050900044832B6CA64A1B0600F13A83AB6CA44AEE
:1050A000180600F130832B6DA14A190600F16483C4
:1050B000AB6D9F4A1B0600F15A832B6E9C4A180663
:1050C00000F15083AB6E9A4A190600F146832B6FAC
:1050D000974A1B0600F13C83AB6F954A180600F116
:1050E0003283D5F88030924A190600F12683D5F82C
:1050F00088308F4A1B0600F11A83D5F890308C4A0D
:10510000180600F14483D5F89830894A190600F151
:10511000388300230193874B0293874B0393874B7C
:105120000593DFF860A2864BDFF85C920493029B44
:10513000186830B1D0F80480FFF7E4FA4046002840
:10514000F8D1039B1868029B1A4600231360019B49
:105150001A4600234AF8223030B1D0F80480FFF715
:10516000D1FA40460028F8D1039A049B1146002248
:105170000A60059A1B781146002241F8042B019A17
:105180000591023B4FF0000129F81210032B00F2A9
:105190003F81DFE813F08B0139018B013901BCF14C
:1051A000400F18BF0023B5E6664A0F78487817709D
:1051B00050708F78C8789770D07010680F79177119
:1051C00086284F7989799171577108BF5E4A5F4F80
:1051D00004BF0F2111705E4A38781178002881F0E1
:1051E000010E41F0020182F800E00CBF8822C822C3
:1051F00045F8312005EBC10180F001000022387034
:105200004A609BE642F221239A4240F0E781DFF8B0
:105210007C91504B504A9EF80200D9F800E0C3F848
:1052200000E00191CDF808C010700021029B0391AD
:105230008A4689460846464A92F800E04EF0020C3B
:1052400005EBCC08002BC8F804000CBF8820C82050
:1052500040EA0A0A9DF8043045F83CA08EF00100AF
:105260003B701070DFF8C8C0DFF8E080DFF8E0A026
:10527000002940F02E81B9F1400F1DD140F002000D
:1052800005EBC005039B6B60019DDFF8A4C0002DFA
:1052900040F036810D0445F088084CF830809DF8C8
:1052A00008503D7082F800E00B44402904D10021F1
:1052B0002A4ACBF800301180294A0123137040E6B6
:1052C00000F0BCFD8BE51A4B254821491A614FF0CF
:1052D000020E80F800E0234F0A702349196099609C
:1052E000224E234D234C9A610D213970FF213170DC
:1052F000DFF89CE0297022701F4D204A8EF80010C4
:105300009F27012406F8047C5D600470DA6007B012
:10531000BDE8F08F1A4A47F83B0013780133137049
:105320003FE543F82500DFF85CA020E5AC9E0220B5
:1053300000800220249E0220789E0220889E022067
:10534000B09E0220B0A00220359E0220349E022092
:10535000A09E0220B8A0022028A00220E09D0220EA
:1053600094200740C0200740880040008820074064
:105370008020074098200740E49D0220389E0220AC
:10538000A19E0220D09D0220A8A00220C09C022045
:105390008C200740535D032B00F2CC8001A151F813
:1053A00023F000BFA34D0000A34D000003540000F4
:1053B000FD530000BE49BF4B80220D2008701A70BB
:1053C000AA077FF500AEF7E540F202339A4240F0BB
:1053D000FC80BEF8042002F07F02042A72D8BEF8D6
:1053E0000230002B6ED1B249019392001144CDF8E6
:1053F00008C00A7842F002020A7016E701235355EA
:10540000CFE400235355CCE4049B4FF001021A7003
:10541000029A019B04320292039A04320392049A84
:1054200001330132042B019304927FF480AEDFF844
:10543000B492DFF8B4A299F800309F4A00218AF8AC
:10544000001013701B0700F10A8199F801309B4A84
:10545000DFF89882137018074FF000022A63AA63DE
:1054600000F1E88099F80230954ADFF880821370E5
:1054700019074FF000022A65AA6500F10381914ADD
:1054800099F80330137000222A67AA671A07DFF819
:105490005C9200F1B8803B780293002283F0010314
:1054A0000193C5F89020C5F89820BEE6049B4FF004
:1054B00000021A70ACE7BEF8042002F07F02042A52
:1054C00040F291807A4B0F221A707F4A01231370A9
:1054D00037E540297FF6D2AE40F002000CEBC00267
:1054E000039B5360019AC2B1784A9DF8085088F82E
:1054F000005040398AF800E040334CF83020D7E6BD
:105500009DF808303B700D04039B82F800E045F0E5
:10551000C8050B444CF83050C7E69DF8083088F8B1
:105520000030039B6A4A8AF800E0403940334CF867
:105530003020BDE618F0080F0CBF0223032353559B
:105540002FE464484FF0020C01704170BEF8061061
:10555000614580F06181604A92F800E04EF0020CF3
:1055600005EBCC034029894628BF4FF0400958601D
:1055700000EB09030393002301930123C9EB01010D
:105580004FEA094A0293C82062E6544B5868002843
:1055900098D0BEF80210BEF804C003E00C3358687F
:1055A00000288FD01A888A42F8D15A886245F5D1EE
:1055B000090A03290CBF90F800C0B3F808C0C5E77A
:1055C000474B44481B780370C0E7B2F5A06F7FF4E7
:1055D00079AF002301930123029326E642F221339F
:1055E0009A42F6D06EE7BEF80230002B7FF46AAF25
:1055F0002F49019392001144CDF808C00A7822F097
:1056000002020A7011E6FFF75FF8002800F0D08070
:1056100008302F4BC9F88400C9F88030FFF754F8E0
:10562000002800F0BD800830284BC5F88C00C5F874
:10563000883030E7FFF748F8002800F0D6800830BF
:10564000234BC8F84400C8F84030FFF73DF8002865
:1056500000F0C48008301D4BE864AB6402E7FFF73C
:1056600033F8002800F0B3800830194B68622B62D1
:10567000FFF72AF8002800F0A3800830134BE862F7
:10568000AB62E2E6FFF720F8002800F0BD800830AA
:105690000F4BC8F86400C8F86030FFF715F8002811
:1056A00000F0AB800830094BE866AB66E7E600BF68
:1056B000C020074080200740C4200740C820074082
:1056C000CC200740D020074094200740C80040006D
:1056D00088004000A49E0220A09E0220DC810000E1
:1056E000AC9E0220D8810000A19E022000800220F2
:1056F000D06A0838FFF706F8C1E4D9F82400083862
:10570000FFF700F8B6E4D06C0838FEF7FBFFCAE4F8
:10571000506C0838FEF7F6FFC0E4D06B0838FEF78F
:10572000F1FFB6E4506B0838FEF7ECFFACE4D2F8BA
:105730008C000838FEF7E6FFDFE4D2F88400083872
:10574000FEF7E0FFD3E4D06F0838FEF7DBFFC8E4D4
:10575000506F0838FEF7D6FFBEE4D06E0838FEF76B
:10576000D1FFB4E4506E0838FEF7CCFFAAE4D06D48
:105770000838FEF7C7FFA0E4506D0838FEF7C2FFF7
:1057800096E4D2F89C000838FEF7BCFFC1E4D2F8DA
:1057900094000838FEF7B6FFB5E44FF0020CD5E6EA
:1057A0009AF80030C5F8880001338AF8003072E6B4
:1057B0009AF80030C9F8800001338AF800302DE7EC
:1057C0009AF80030A86201338AF800303DE69AF872
:1057D0000030286201338AF8003049E79AF8003037
:1057E000A86401338AF800303CE69AF80030C8F823
:1057F000400001338AF8003027E79AF80030A866A5
:1058000001338AF800303AE69AF80030C8F86000B0
:1058100001338AF8003040E7BCF1400FE14628BF71
:105820004FF0400900EB0903039300230193012388
:10583000C9EB0C014FEA094A0293FCE42DE9F0415F
:10584000FFF7C4F82F4C304B3048DFF8D880304F8A
:10585000304D314EDFF8D0C0DFF8D0E000221A60C2
:105860005A609A60DA601A615A619A61DA611A6262
:105870005A629A62DA621A635A639A63DA631A6442
:105880005A649A64DA641A655A659A65DA651A6622
:105890005A669A66DA661A675A679A67DA67C3F8C9
:1058A00080202168C3F8842041F4802121600168B0
:1058B00041F040710160C3F3072188F8001004F53E
:1058C0002834C3F307411B0E3970CC342B7000F120
:1058D0002040FF238CF80030104D8EF8003000F689
:1058E000041033700E49012308F8083C702622701A
:1058F0004FF40014102207F82C3C2E7004600A703C
:10590000BDE8F081348004400080022000D80040CF
:10591000B0200740B42007401020074035E400E0E5
:10592000082107409C20074080200740882007402E
:10593000054B1878054B1A78C0B2D3B2984238BFDD
:105940004030C01A704700BF229F0220B99E02203B
:1059500010B5284B1A79920620D52749DA790B78A9
:105960002648013300783F2BC8BF0023834218BF6D
:105970002348D2B21EBFC254DAB20A70214A11685B
:1059800061B1214A1278D2B2934236BFC2F14002CD
:105990009B1A9B18272BC4BF01230B701549CA788B
:1059A000D2B2140616D50B79180613D5174B164C20
:1059B00018782378DBB2984202D16C23CB7009E0CF
:1059C0000133282B28BF00231148C05CDBB2C0B2D2
:1059D000C871237051060CD5064B1A79520608D5AA
:1059E0000C4A002111700C4A126802B111702C226D
:1059F000DA7010BD00D00640229F0220B99E02201E
:105A0000E29E0220B49E0220239F0220289F0220B3
:105A1000BA9E0220B89E0220249F0220054B1878CF
:105A2000054B1A78C0B2D3B2984238BF4030C01A82
:105A3000704700BF9A9F0220319F0220F0B5344981
:105A40000B7913F0300F2FD072B68B7D03F0FF046B
:105A500023B9CB7940234B7462B625E062B62D485A
:105A60002D4A037812782D4FDBB2D2B20546581C6E
:105A70004028CE7928BF00209042F6B21CBF3E5489
:105A80000346601E10F0FF04F1D1D9B229702449F9
:105A9000096849B1934236BFC2F140029B1A9B1874
:105AA000272BC4BF01230B70194AD178C9B20D0648
:105AB0001ED513791C061BD51A4B1B481D7803787D
:105AC0001A4EEDB2DBB2AB420AD00133282B28BF0D
:105AD00000231479F45CE4B2D471147D072CF2D95C
:105AE000DBB203700A4B1A79100644BF7C22DA70CD
:105AF00049060CD5064B1A79520608D50C4A0021E6
:105B000011700C4A126802B111703C22DA70F0BDBB
:105B100000B006409A9F0220319F02205A9F022027
:105B20002C9F0220A09F02209B9F0220329F0220D8
:105B3000309F02209C9F022010B5204B2048214915
:105B400060221A70E1225A701F4B204A1C78204BA9
:105B5000082C01D1012402E00A2C03D1392404606D
:105B6000132005E00C2C0CBF35243D2404601220CA
:105B7000086014601860174B17491B78174A03B167
:105B800001230B601360164B164A1978164B012936
:105B900001D880210BE0042901D8842107E00829DD
:105BA00001D8852103E0102994BF86218721116047
:105BB00019600E4B01221A7010BD00BF0040074053
:105BC00008B003400CB00340E687022008B00B4049
:105BD0000CB00B40A29F022020B0034020B00B402D
:105BE000E787022024B0034024B00B40A19F02208D
:105BF000054B1878054B1A78C0B2D3B2984238BF1B
:105C00004030C01A704700BF12A00220A99F022096
:105C100010B5284B1A79920620D52749DA790B78E6
:105C20002648013300783F2BC8BF0023834218BFAA
:105C30002348D2B21EBFC254DAB20A70214A116898
:105C400061B1214A1278D2B2934236BFC2F140020A
:105C50009B1A9B18272BC4BF01230B701549CA78C8
:105C6000D2B2140616D50B79180613D5174B164C5D
:105C700018782378DBB2984202D16C23CB7009E00C
:105C80000133282B28BF00231148C05CDBB2C0B20F
:105C9000C871237051060CD5064B1A79520608D5E7
:105CA0000C4A002111700C4A126802B111702C22AA
:105CB000DA7010BD00A00E4012A00220A99F0220A1
:105CC000D29F0220A49F022013A0022018A002202D
:105CD000AA9F0220A89F022014A0022010B5104CF9
:105CE00023686BB1206843885A1C03441C7A0388DC
:105CF0009A4212D3FEF706FD094B00221A600DE00E
:105D0000084B1B7813B94FF0FF3010BD0320FEF78E
:105D100023FF20600028E5D1F5E74280204610BD32
:105D200024A00220AC9E0220044B9888044B1A68E1
:105D30001AB1138852889B1A18447047A8A00220F1
:105D400024A002202DE9F84F314DDFF8D490012333
:105D500082460C462B700E464F46002E53D0D9F883
:105D600000303BBBDFF8B0B047F20958294B1B7835
:105D700003F0FF010BB9297015E00420FEF70AFFBC
:105D8000072807D801232B70FEF79EFC386088B9DE
:105D90001F4B1870B8F1010802D09BF8003033B1E6
:105DA0001D4B01221A704FF0FF30BDE8F88F00F054
:105DB00039F9DBE7184B0021197039684B88C3F1BA
:105DC0004000B04228BF304603EB000E0B44A1F860
:105DD00002E0361A07330AEB0008C24504D01AF86D
:105DE000010B03F8010FF8E74B883F2B06D940233E
:105DF0000B800420FEF748FF00233B60074B052281
:105E00001A70C246A9E72E702046BDE8F88F00BF81
:105E10001AA00220AC9E022020A0022019A002207D
:105E20001CA0022007B502AB012103F8010D1846A2
:105E3000FFF788FF03B05DF804FBFFFF38B50E4B9A
:105E40001B7803F0FF05ABB90C4C216831B14B88CE
:105E50000B800420FEF718FF256038BDFEF734FCE8
:105E6000014620B10420BDE83840FEF70DBF044BC9
:105E700001221A7038BD00BF1AA002201CA0022007
:105E800019A002207047EFF3108072B6B0FA80F0CC
:105E90004009704700B162B67047FFFFF8B50C4E7D
:105EA0000C4F0025FFF7EFFF346802466CB16369C1
:105EB00033600BB19D6100E03B601046FFF7EAFFE5
:105EC0006577A36820469847ECE7FFF7E3FFF8BD46
:105ED0002CA0022030A00220FFF7E0BF15490B687C
:105EE00030B513B98360C36009E004681A6894424E
:105EF00007D20025121B8360C560D8601A60086055
:105F000015E002681C689968121B026061B10C6898
:105F1000A2420B46F5D28160C968C160D860C168F1
:105F2000A21A88601A6002E08160C3609860022350
:105F3000037530BD34A0022070B5164D2C680026C4
:105F4000BCB1236813B1013B236012E0A26802B127
:105F5000D36020692A60036826751B6822460021E9
:105F6000984763681BB123602046FFF7B7FF2C6892
:105F7000E6E7FFF788FF084B00221C681A60FFF76E
:105F800089FF2CB1A5682046FFF7A8FF2C46F8E74B
:105F900070BD00BF34A0022044A00220024A136852
:105FA00001331360FFF7C8BFC09C02207047FFFF9A
:105FB000164AF8B51368164D43F080731360154AFE
:105FC000136843F001031360134B2E681C688CB1F7
:105FD000237A6BB123682F681B68204698472A688C
:105FE000E388D21B120991B29A42A18088BFE18056
:105FF0006469ECE72B68094A9B1B1B0999B2118065
:10600000074A1088834288BF1180F8BDFCED00E08C
:10601000041000E0001000E048A002204EA0022082
:106020004CA0022038B5254C2378002B45D1012304
:106030002370FFF779FE08B1FFF7B8FFFEF7FEFC0B
:1060400008B1FFF71FFFFFF7E9FC08B100F090FB74
:10605000FEF7C4FA08B100F03AF8FFF769FC08B19E
:1060600000F04CF8FFF7C4FD08B100F048F8FEF767
:1060700037FC08B100F02AF800232370EFF3058302
:10608000DBB9EFF3108272B60D4D286810B10D4CDC
:10609000217811B18AB962B638BD012323704369F2
:1060A0002B600BB1996101E007490B6002B962B640
:1060B0000025457783689847257038BD50A0022099
:1060C0003CA0022040A0022038A002207047704768
:1060D00010B5044600F04EFB204610BD0448054AAA
:1060E0000549002303608023037100F08DBB00BFCE
:1060F00054A00220F8860220D1600000704770474B
:10610000054A40F243434FF4886113605360916045
:10611000D36013615361704700D00440054A40F2D8
:1061200003130021136053609160D36013615361C6
:10613000704700BF00D004404FF47A7330B51B4C59
:106140005843012209231101B4FBF1F1884203D322
:1061500001241346154907E0013BF9D05200F2E74C
:10616000102C134404D00134B1FBF3F5A842F7D34B
:106170000F48036823F008030360016821F47F23BC
:10618000D20123F47F6343F4602302F47F421A4375
:10619000631E42EA0313074A036013681B07FCD51A
:1061A000036843F00803036030BD00BF006CDC02ED
:1061B0002C100B4024100B401E4A136843F0800340
:1061C00010B513601C4B1C461968C907FCD4216824
:1061D0008907F9D4194B4FF080711860146818487A
:1061E000144B2040013910B90029F7D102E009B160
:1061F000012807D0136843F4702343F001031360B0
:10620000012010BD1A68120605D51A6842F0011265
:106210001A60032010BD18681A6810F4803017BF88
:1062200042F0011242F0010205201A6008BF1A6014
:1062300010BD00BF30100B4024100B400C100B4061
:1062400001000E00F8B50A4D0A4F4FF47A7400268B
:106250002E600948FFF7B0FF013C05D03B685B07A3
:1062600005D50028F4D0F8BD002808BF0520F8BDEA
:1062700008100B4024100B400000DB0C70B5084DDB
:10628000002306462B600748FFF796FF38B9064CF7
:10629000064823682E60FFF78FFF00B9236870BDA2
:1062A00008100B4000001A3710100B4000000229A4
:1062B000074B1A783AB99A783AB15B78002B0CBF41
:1062C000022003207047002070470120704700BF64
:1062D0005CA0022070B5384B1A780546002A68D1B8
:1062E0005B7803B94902354C35484FF6FF7323609C
:1062F000344B4FF48132196043F8042CFFF75CFFF4
:10630000002857D1304B3148314A1B6805F1400312
:1063100005F51075216841F0200611F4E00F2660A4
:1063200009D041F4E003254A43F020031360FFF74E
:1063300089FF012036E001680905FCD5116843F8A2
:10634000401C116843F83C1C116843F8381C116864
:1063500043F8341C116843F8301C116843F82C1CB6
:10636000116843F8281C116843F8241C116843F88D
:10637000201C116843F81C1C116843F8181C116894
:1063800043F8141C116843F8101C116843F80C1CE6
:10639000116843F8081C116843F8041C4033AB42F1
:1063A000B8D1002023689B07FCD5044B094A1A602A
:1063B00070BD032070BD00BF5CA0022030100B40F8
:1063C00010003A1108100B4010100B4024100B4025
:1063D00020100B4022000001F8B5294B1A78054621
:1063E000002A4AD15B7803B94902264C2648236823
:1063F0002360264B4FF48132196043F8042CFFF7D9
:10640000DBFE00283AD1224BDFF88CE01B6805F553
:106410000076274623681B4AD906FBD53B6813F450
:10642000E00F06D0136843F4E00343F01003136059
:1064300016E005F1400255F8043BCEF80030AA42C0
:10644000F9D123680F4943F010032360206810F44A
:10645000E00009D00B6843F4E00343F010030B6045
:10646000FFF7F0FE012001E0B242D3D123689B0781
:10647000FCD5044B074A1A60F8BD0320F8BD00BFE5
:106480005CA0022030100B4000003A1808100B40AE
:1064900010100B401200000120100B40064A136838
:1064A00043F04063136002F56A323032136843F4FC
:1064B00000331360704700BF00D800402DE9F0475B
:1064C000934CFFF7EBFFFFF729FE236843F080733F
:1064D00043F4004323602368DE01FCD44FF4C8700A
:1064E000FFF72AFE8B4A13689D07FCD1FFF708FED1
:1064F000894B8A4E8A494FF481321A603368894A3F
:1065000023F0380343F02803336013681360864B8D
:10651000196040F2DC53216841F00061216021687C
:106520000901FCD4013BF6D11168804C41F0800197
:106530001160784A1268636012F4803F14BF002033
:10654000022020706370A370A360002840F0DD80FB
:10655000774A784F136018463B60FFF72DFE50B91D
:10656000754D76482B684FF4D5733B60FFF724FEDA
:1065700028B105280AD001202070BDE8F0872B68DB
:106580002B68B3F5D57FF6D1012363700020FFF7A8
:1065900075FE0028EFD12B6813F4401F20D06378DC
:1065A000DFF8A0A1002B664B0CBF4FF440199946B1
:1065B00080464846FFF762FE002840F0A0802B6826
:1065C000002B08F1010802DBD045F2D19AE05D4BC7
:1065D000984500F09780584B1B685B0040F1928013
:1065E00000233B605848DFF84C91FFF7E5FD002899
:1065F000C1D12B68C9F800005448DFF83C81FFF78F
:10660000DBFD0028B7D1D8F80030D8F8003050486A
:10661000DFF818811B0C1B046360C9F80030FFF71A
:10662000CBFD0028A7D14B4A4B4813681B0E88F8B6
:1066300003304A4B1B6813F4400F14D113681168E0
:1066400002680068890201F4406141EA9252511CDB
:10665000C0F3C2120232C3F3032301FA02F2093B70
:1066600002FA03F307E0012388F802300368C3F35A
:10667000152301339B02C8F8083063683B60384833
:10668000DFF8A880DFF8AC90FFF796FD00287FF4D4
:1066900072AF2B683348284F4FF40073C9F80030AD
:1066A000FFF78AFD00287FF466AF3B68D8F8043016
:1066B000C9F800302C48FFF77FFD00287FF45BAF5E
:1066C0003B682A480223C9F80030FFF775FD00280F
:1066D0007FF451AF3B68336823F0060333603368BF
:1066E00043F002033360FFF719FD46F2A810FFF7ED
:1066F00023FDFFF705FD98F80000BDE8F0870120B5
:10670000BDE8F087002363706AE7BDE8F08700BF4B
:106710002C100B4024100B4004100B4028100B4091
:10672000BB007F1130100B4034100B405CA00220E6
:1067300038100B4008100B4010100B4000001A08D6
:1067400000003040A08601000000090200001A038A
:106750000000090918100B4014100B401C100B40CE
:1067600000001B0700001A1000001A3700001A066C
:1067700070477047016830B5A1B10B4B0B441B113A
:1067800003F130025511012402F01F0204FA02F253
:10679000064C44F82520064A064C42F823400023C4
:1067A0008B60036030BD00BF008FFCBF80E100E064
:1067B000E887022073670000024B01221A60024B37
:1067C0001B6818470C710340E8870220024B012226
:1067D0001A60024B5B6818471C710340E88702206F
:1067E000024B01221A60024B9B6818472C71034030
:1067F000E8870220024B01221A60024BDB6818472F
:106800003C710340E88702200B460146184600F021
:1068100001B800BF13460A460146022000F02EBD13
:10682000014B1868704700BF208C022070B50F4ED6
:106830000F4D761BB61018BF002405D0013455F853
:10684000043B9847A642F9D10A4E0B4D761B01F046
:10685000F1FCB61018BF002406D0013455F8043BF3
:106860009847A642F9D170BD70BD00BF40820000BC
:10687000408200004C82000040820000024B014632
:10688000186800F00BB800BF208C0220024B0146B4
:10689000186800F0B7BD00BF208C02202DE9F04F32
:1068A00001F10B05162D83B0064640F29F8035F0AE
:1068B000070500F1BF80A94200F2BC8000F08EFB0A
:1068C000B5F5FC7FC0F09C826B0A00F0BA80042B07
:1068D00000F28381A80900F1390E4FEA4E033830E7
:1068E000C44F07EB8303A3F108015C68A14207D101
:1068F000ACE0002A80F2AC80E468A14200F0A680FF
:10690000636823F003035A1B0F2AF2DDB9493C697F
:1069100001F1080E744500F0B381636823F00303AE
:106920005A1B0F2A00F39981002AC1F814E0C1F81C
:1069300010E080F29E80B3F5007F80F06781DB0875
:1069400003F1010C01229B1002FA03F34A6851F88B
:106950003C80C4F8088001EBCC091A43A9F1080374
:10696000E3604A6041F83C40C8F80C4083100124C1
:106970009C40944200F28A80144206D120F0030029
:106980006400144200F10400FAD007EBC009CC46C1
:106990008046DCF80C108C4507D173E1002A80F2A8
:1069A0008181C9688C4500F06D814B6823F0030339
:1069B0005A1B0F2AF2DD0C46D1F80CC054F8088F90
:1069C0004B1945F001054D6042F00101C8F80CC0BB
:1069D0003046CCF808807B613B61C3F80CE0C3F81B
:1069E00008E059609A5000F0FBFA1FE0102921D806
:1069F00000F0F4FA1025062302207E4F07EB8303F4
:106A0000A3F108025C68944200F045816368E16884
:106A1000A56823F00303234430465A68E96042F036
:106A200001028D605A6000F0DBFA0834204603B0A2
:106A3000BDE8F08F00240C232046336003B0BDE88E
:106A4000F08F80234FF0400E3F2049E770465DE70E
:106A50002344E1685A68A56842F00102E9603046C3
:106A60008D605A6000F0BCFA0834204603B0BDE8DF
:106A7000F08F234430465A6842F001025A6000F019
:106A8000AFFA0834204603B0BDE8F08FBC686368F5
:106A900023F00308A84504D3C5EB08030F2B00F32C
:106AA0008C80554BDFF860911A68D9F800300133BB
:106AB0002A4404EB080A00F0608102F580520F328C
:106AC00022F47F6222F00F0211463046019200F05C
:106AD00089FAB0F1FF3F8346019A00F05881824560
:106AE00000F2FC80454B1968DA451144196000F04A
:106AF0005381D9F80000DFF810E101301BBFCAEB69
:106B00000B0A5144CEF800B019601BF0070100F0E9
:106B10001781C1F10800C1F58051834408315A44FE
:106B2000C2F30B02C2EB010949463046019300F063
:106B300059FA431C019B00F03F81CBEB00024A4411
:106B400042F001021968C7F808B04944BC42CBF8CA
:106B500004201960DFF8A49016D0B8F10F0F40F2AE
:106B6000FD806268A8F10C0323F00703E01802F02F
:106B700001024FF0050E1A430F2B6260C0F804E0CB
:106B8000C0F808E000F21C811D4BBC681A689142F5
:106B900088BF19601B4B1A689142626888BF1960F0
:106BA00022F003029542A2EB050301D80F2B04DC6F
:106BB000304600F015FA002438E7621943F001036B
:106BC00045F0010565603046BA60536000F008FA90
:106BD0000834204603B0BDE8F08F142B71D9542B34
:106BE00000F2A480280B00F16F0E4FEA4E036E30C6
:106BF00076E600BF248C022074A0022078A0022038
:106C000070A002206CA00220309002205A0A042AB0
:106C10005ED9142A00F2B38002F15C0149005B32B4
:106C200007EB810C57F82110DFF8DC81ACF1080C80
:106C30008C4500F088804A6822F00302934202D219
:106C400089688C45F7D1D1F80CC07A68C4F80CC0BB
:106C5000A160CCF80840CC6088E6631942F00107D7
:106C600045F00105656030464B610B61C3F80CE0EF
:106C7000C3F808E05F609A50083400F0B1F9D5E637
:106C80004A6873E608F1010818F0030F0CF1080CCC
:106C90007FF47FAE30E0DC68A34208BF02303FF4EF
:106CA00035AEB3E60B440C465A68C96854F8085F21
:106CB00042F001025A603046E9608D6000F090F9C0
:106CC000B4E603F15C0E03F15B004FEA4E0307E606
:106CD0009A0902F1390149003832A1E7BC424A4B16
:106CE0003FF400AF9C68626822F003025AE759F84B
:106CF0000839994540F0828010F0030F00F1FF3011
:106D0000F5D17B6823EA04037B6064009C423FF674
:106D1000BDAE002C3FF4BAAE1C4240467FF435AE07
:106D200064001C4200F10400FAD02EE6B3F5AA7FFD
:106D300018D8E80B00F1780E4FEA4E037730CFE514
:106D40004FF48051EBE60121D8F80430921001FA9B
:106D500002F21A43C8F80420614677E70123CBF812
:106D6000043025E740F25452934220D8A80C00F199
:106D70007D0E4FEA4E037C30B2E51032A4E6542A71
:106D800026D81A0B02F16F0149006E3248E7BC6841
:106D9000626822F0030205E7CAF30B0000287FF4C3
:106DA000A8AE4244BB6842F001025A60ECE6FE2302
:106DB0004FF07F0E7E2093E501224FF00009C1E6DF
:106DC00004F10801304600F01DFBD9F80010DBE6A5
:106DD000B2F5AA7F05D8DA0B02F1780149007732C3
:106DE0001EE740F254518A4205D89A0C02F17D0107
:106DF00049007C3214E7FE217E2211E77B6884E79C
:106E0000E808431C5B00F8E5248C0220844641EA34
:106E1000000313F003036DD1403A41D351F8043B12
:106E200040F8043B51F8043B40F8043B51F8043B64
:106E300040F8043B51F8043B40F8043B51F8043B54
:106E400040F8043B51F8043B40F8043B51F8043B44
:106E500040F8043B51F8043B40F8043B51F8043B34
:106E600040F8043B51F8043B40F8043B51F8043B24
:106E700040F8043B51F8043B40F8043B51F8043B14
:106E800040F8043B51F8043B40F8043B51F8043B04
:106E900040F8043B51F8043B40F8043B403ABDD273
:106EA000303211D351F8043B40F8043B51F8043B15
:106EB00040F8043B51F8043B40F8043B51F8043BD4
:106EC00040F8043B103AEDD20C3205D351F8043BA4
:106ED00040F8043B043AF9D2043208D0D2071CBF70
:106EE00011F8013B00F8013B01D30B880380604699
:106EF000704700BF082A13D38B078DD010F003030F
:106F00008AD0C3F10403D21ADB071CBF11F8013B7E
:106F100000F8013B80D331F8023B20F8023B7BE7CD
:106F2000043AD9D3013A11F8013B00F8013BF9D2F8
:106F30000B7803704B7843708B7883706046704792
:106F400070B4840746D0541E002A41D0CDB2034607
:106F500002E0621EE4B3144603F8015B9A07F8D11D
:106F6000032C2ED9CDB245EA05250F2C45EA05455F
:106F700019D903F110022646103E0F2E42F8105C7C
:106F800042F80C5C42F8085C42F8045C02F1100222
:106F9000F2D8A4F1100222F00F0204F00F04103214
:106FA000032C13440DD91E462246043A032A46F800
:106FB000045BFAD8221F22F003020432134404F0C7
:106FC00003042CB1C9B21C4403F8011BA342FBD13A
:106FD00070BC704714460346C2E700BF704700BF4D
:106FE000704700BF38B5074C0023054608462360AC
:106FF000F9F750FC431C00D038BD2368002BFBD0B0
:107000002B6038BDBCA0022080EA0102844612F049
:10701000030F4FD111F0030F32D14DF8044D11F091
:10702000040F51F8043B0BD0A3F101329A4312F044
:10703000803F04BF4CF8043B51F8043B16D100BF1D
:1070400051F8044BA3F101329A4312F0803FA4F1AE
:1070500001320BD14CF8043BA24312F0803F04BF35
:1070600051F8043B4CF8044BEAD023460CF8013BA2
:1070700013F0FF0F4FEA3323F8D15DF8044B70474C
:1070800011F0010F06D011F8012B0CF8012B002A8A
:1070900008BF704711F0020FBFD031F8022B12F079
:1070A000FF0F16BF2CF8022B8CF8002012F47F4F34
:1070B000B3D1704711F8012B0CF8012B002AF9D13C
:1070C000704700BFFFFFFFFFFFFFFFFFFFFFFFFF56
:1070D000FFFFFFFFFFFFFFFFFFFFFFFFFFFFFFFFC0
:1070E000FFFFFFFFFFFFFFFFFFFFFFFFFFFFFFFFB0
:1070F000FFFFFFFFFFFFFFFFFFFFFFFFFFFFFFFFA0
:1071000090F800F06DE9024520F007016FF0000CE7
:1071100010F0070491F820F040F049804FF000048F
:107120006FF00700D1E9002391F840F000F108006A
:1071300082FA4CF2A4FA8CF283FA4CF3A2FA8CF3A2
:107140004BBBD1E9022382FA4CF200F10800A4FA09
:107150008CF283FA4CF3A2FA8CF3E3B9D1E904235D
:1071600082FA4CF200F10800A4FA8CF283FA4CF394
:10717000A2FA8CF37BB9D1E9062301F1200182FA4E
:107180004CF200F10800A4FA8CF283FA4CF3A2FA54
:107190008CF3002BC6D0002A04BF04301A4612BA62
:1071A000B2FA82F2FDE8024500EBD2007047D1E965
:1071B000002304F00305C4F100004FEAC50514F0F4
:1071C000040F91F840F00CFA05F562EA05021CBFC5
:1071D00063EA050362464FF00004A9E7002A41D0A4
:1071E00040EA010313F00303F0B425D1032A23D9A5
:1071F00004680D68AC421FD1043A35D0A4F10135C2
:1072000025EA040414F0803F31D1071D0D1D0DE067
:1072100057F8043B0E68A3F10134B34224EA030497
:107220000AD1043A20D014F0803F23D1032A294602
:10723000384605F10405EBD803780C789C4202F13E
:10724000FF320CD182B114B916E06AB17BB110F8EB
:10725000013F11F8014FA34202F1FF32F5D0181B94
:10726000F0BC7047104670471046F0BC7047184697
:10727000F0BC70470020F3E72046F1E72DE9F04726
:10728000254C2568D5F848410646884692469946D9
:10729000C4B360681F2817DC431C76B104EB80057B
:1072A0000122C5F888A0D4F8881182401143022E2B
:1072B000C4F88811C5F808911ED00230636044F804
:1072C00020800020BDE8F087144B03B34FF4C87052
:1072D000FFF7D4FA0446D0B1D5F84831002780E84A
:1072E0008800C5F8484138460123C4F88871C4F8BD
:1072F0008C71002EE1D0D1E7D4F88C110A43C4F888
:107300008C21DAE705F5A674C5F84841C1E74FF0CE
:10731000FF30BDE8F08700BF308200007D680000CC
:10732000024B13B1024800F005B87047000000009E
:1073300041730000002301461A461846FFF79EBF1E
:1073400038B5074D074C2C1BA41005D0013C55F84F
:10735000043D9847002CF9D1BDE8384000F076BFD5
:107360000000000000000000F8B5234F0C46064660
:10737000FFF734FEBB685D6825F00305291B01F6A5
:10738000EF7121F47F6121F00F01A1F58054B4F574
:10739000805F07DB00213046FFF724FEBB682B44EB
:1073A000984204D03046FFF71BFE0020F8BD614232
:1073B0003046FFF717FE01300DD0104BBA68196840
:1073C0002D1B45F001053046091B55601960FFF77C
:1073D00007FE0120F8BD00213046FFF703FEBA6822
:1073E000831A0F2BDEDD064C0449246843F00103A9
:1073F000001B53600860D5E7248C022078A002208F
:1074000030900220002945D02DE9F0410D468046FC
:10741000FFF7E4FD55F8047C6A4927F00103A5F164
:107420000804E2188E685068B24220F0030062D06F
:10743000FE0750600BD455F8087CE41B01F1080EE0
:10744000A56875453B446FD0E768EF60BD601518CF
:107450006D68ED0742D543F001026260E350B3F579
:10746000007F18D2DB085A1C4D6851F83270A760B3
:1074700001209B1000FA03F301EBC2001D43083802
:10748000E0604D6041F83240FC604046BDE8F041AC
:10749000FFF7A6BD70475A0A042A53D89A0902F189
:1074A00039077F0002F1380501EB870051F82720EA
:1074B0004449083890424DD0516821F003018B4275
:1074C00002D292689042F7D1D068E060A2608460F6
:1074D000D4604046BDE8F041FFF782BD95683A4F61
:1074E000BD4203443FD0D068E86043F001028560AC
:1074F0006260E350B3E7FF07034407D455F8082C54
:10750000A41A1344A068E268C26090602F4A12680F
:1075100043F00100934260608C60B6D32C4B404630
:107520001968FFF721FFB0E711184968C90744D46B
:107530009168D268CA60034443F0010091606060C2
:10754000E350A2E7142A17D802F15C077F0002F18A
:107550005B05A9E7AA104B68012505FA02F213435F
:107560004B600246B1E743F001024C610C61E560FB
:10757000A5606260E35088E7542A06D81A0B02F12E
:107580006F077F0002F16E058EE7B2F5AA7F06D87D
:10759000DA0B02F178077F0002F1770584E740F209
:1075A0005450824206D89A0C02F17D077F0002F106
:1075B0007C0579E7FE277E2576E743F001026260CD
:1075C000E35062E7248C02202C8C02202C900220B5
:1075D00074A0022048415244204641554C54004278
:1075E0005553204641554C54004D454D4F5259205E
:1075F0004D414E4147454D454E54204641554C5412
:10760000005553414745204641554C5400554E4B7B
:107610004E4F574E204641554C54000A0A5265675A
:1076200069737465722076616C756573206174206E
:1076300074696D65206F66206661756C743A0A0026
:1076400020205230202020203A2030782530386CFD
:10765000780020205231202020203A203078253018
:10766000386C780020205232202020203A203078B8
:107670002530386C780020205233202020203A20FA
:1076800030782530386C780A0020205231322020A2
:10769000203A2030782530386C780020204C522059
:1076A0002020203A2030782530386C780020205077
:1076B00043202020203A2030782530386C78002074
:1076C000205053522020203A2030782530386C78D2
:1076D0000020205350202020203A203078253038B8
:1076E0006C780A0020204346535220203A203078FC
:1076F0002530386C780020205546535220203A20FF
:1077000030782530386C78002020484653522020AD
:107710003A2030782530386C780020204446535287
:1077200020203A2030782530386C780020204246DE
:10773000415220203A2030782530386C780A0020D9
:10774000204343522020203A2030782530386C786E
:107750000020204146535220203A203078253038EE
:107760006C780A00537461636B20636F6E74656E8E
:1077700074733A0A0025303858003A20200025302A
:10778000325800207C007C0D0A00525443204E6F7A
:10779000742079657420696D706C656D656E7465B3
:1077A000642E0A0025642F25642F25642025643A61
:1077B00025643A25642E256425640A004B36344638
:1077C00020536F4320436F6E6669677572617469F9
:1077D0006F6E3A0A004F6E2D626F617264204465CD
:1077E00076696365733A0A00202020204652414D95
:1077F00020202020202028253038583A253038589D
:10780000292E0A00202020204652414D4E5620208D
:10781000202028253038583A25303858292E0A009B
:10782000202020204652414D4E564320202028251E
:107830003038583A25303858292E0A002020202088
:1078400052414D2020202020202028253038583A31
:1078500025303858292E0A00202020205344204368
:107860004152442020202844657669636573203D99
:1078700025303264292E0A002020202054494D450D
:107880005231202020202854696D65727320203DDC
:1078900025303264292E0A0020202020494E5452DF
:1078A000204354524C20284368616E6E656C733DD2
:1078B00025303264292E0A00202020205053320A1D
:1078C00000202020205350490A00416464726573EF
:1078D0007365733A0A0020202020435055205265DA
:1078E00073657420566563746F72204164647265B9
:1078F0007373203D20253038580A00202020204373
:107900005055204D656D6F727920537461727420EB
:1079100041646472657373203D20253038580A0035
:1079200020202020537461636B2053746172742093
:10793000416464726573732020202020203D20253F
:107940003038580A004D6973633A0A00202020201D
:1079500053797374656D20436C6F636B2046726559
:107960007120202020202020203D2025642E25303D
:1079700034644D487A0A004B36344658353132006B
:107980001B5B410E101B5B317EFFFFFFC97A0000BD
:1079900001000000D17A000001000000D67A00004A
:1079A000020000001B5B337E1B5B441B30461B5BED
:1079B000347E081B5B420DFFDF7A000001020000ED
:1079C000E07A000001030000E17A000001040000F9
:1079D000E27A000001050000E37A000001060000E1
:1079E000E47A000001070000B27900000101000004
:1079F000E97A000001080000B6790000010B0000E0
:107A0000837900000109000084790000010A000068
:107A100085790000040D0000E57A0000040C0000E8
:107A2000A4790000040E0000AB790000030F0000F1
:107A3000AE790000040F0000D87A000004100000A6
:107A4000EA7A0000041100008079000003120000AF
:107A5000B379000003130000DC7A00000314000077
:107A6000A879000003150000253034642020257318
:107A70000A004661696C656420746F2072657365E5
:107A8000742074686520686973746F727920666900
:107A90006C6520746F20454F462E0A0043616E6E60
:107AA0006F74206F70656E2F6372656174652068F6
:107AB0006973746F72792066696C652C20646973D0
:107AC00061626C696E672E0A00686973746F7279FF
:107AD00000686973740021001B5B357E1B5B4301EA
:107AE00002030405061B5B327E0B1B5B367E010026
:107AF0000400100040000001000200002B2E2C3B6F
:107B00003D5B5D2F5C222A3A3C3E3F7C7F00464134
:107B10005400464154333200222A2B2C3A3B3C3D40
:107B20003E3F5B5D7C7F00EBFE904D53444F5335F1
:107B30002E30004E4F204E414D4520202020464102
:107B4000543332202020004E4F204E414D452020FE
:107B50002020464154202020202000534400809AB9
:107B600045418E418F804545454949498E8F9092C8
:107B7000924F994F555559999A9B9C9D9E9F41496B
:107B80004F55A5A5A6A7A8A9AAABACADAEAFB0B1FD
:107B9000B2B3B4B5B6B7B8B9BABBBCBDBEBFC0C14D
:107BA000C2C3C4C5C6C7C8C9CACBCCCDCECFD0D13D
:107BB000D2D3D4D5D6D7D8D9DADBDCDDDEDFE0E12D
:107BC000E2E3E4E5E6E7E8E9EAEBECEDEEEFF0F11D
:107BD000F2F3F4F5F6F7F8F9FAFBFCFDFEFF01000D
:107BE0000200040008001000200000005B7B000081
:107BF0000000000000000000000000004469736BFA
:107C0000204572726F720A00496E7465726E616C03
:107C1000206572726F722E0A004469736B206E6F5A
:107C2000742072656164792E0A004E6F2066696C5B
:107C30006520666F756E642E0A004E6F2070617449
:107C40006820666F756E642E0A00496E76616C69F5
:107C5000642066696C656E616D652E0A0041636320
:107C60006573732064656E6965642E0A0046696CED
:107C70006520616C726561647920657869737473DD
:107C80002E0A0046696C652068616E646C65206927
:107C90006E76616C69642E0A005344206973207704
:107CA000726974652070726F7465637465642E0AFE
:107CB000004472697665206E756D62657220697325
:107CC00020696E76616C69642E0A004469736B20CA
:107CD0006E6F7420656E61626C65642E0A004E6F73
:107CE00020636F6D70617469626C652066696C6594
:107CF00073797374656D20666F756E64206F6E2086
:107D00006469736B2E0A00466F726D617420616244
:107D10006F727465642E0A0054696D656F75742CFA
:107D2000206F7065726174696F6E2063616E636548
:107D30006C6C65642E0A0046696C65206973206C62
:107D40006F636B65642E0A00496E737566666963BE
:107D500069656E74206D656D6F72792E0A00546FBF
:107D60006F206D616E79206F70656E2066696C653D
:107D7000732E0A00506172616D65746572732069BB
:107D80006E636F72726563742E0A00537563636568
:107D900073732E0A00556E6B6E6F776E206572726C
:107DA0006F722E0A000A256C752062797465732043
:107DB000257320617420256C752062797465732F9A
:107DC0007365632E0A0072656164002530345800C3
:107DD0002020202020202020007A4F53000A2A2A29
:107DE00020257320280030322F30352F32303230AA
:107DF0000076312E30320020435055292025732043
:107E00002573202A2A0A0A006175746F65786563F4
:107E10002E626174007A4F532E6873740046616954
:107E20006C656420746F20696E697469616C697334
:107E300065207364206361726420302C20706C654F
:107E400061736520696E6974206D616E75616C6C1B
:107E5000792E0A00303A002A2000436C656172696D
:107E60006E672E2E2E2E00436F7079696E672E2E50
:107E70002E00436F6D706172696E672E2E2E002585
:107E800030386C782825303878292D3E2530386CEC
:107E9000782825303878290A0044756D70204D65A2
:107EA0006D6F72790A000A436F6D706C6574652E90
:107EB0000A002530385820253032582D003F3F3FEA
:107EC0000A002530385820253034582D0025303808
:107ED0005820253038582D00457865637574696ED3
:107EE0006720636F646520402025303878202E2E6F
:107EF0002E0A0043616C6C696E6720636F646520B5
:107F0000402025303878202E2E2E0A0043616C6CDC
:107F10002072657475726E656420636F64652028D5
:107F20002564292E0A0052657374617274696E6744
:107F3000206170706C69636174696F6E2E2E2E0AF9
:107F400000436F6C64207265626F6F74696E672E98
:107F50002E2E0A0062696E0025643A5C25735C254A
:107F6000732E2573004B36340025643A5C25735C10
:107F700025730025643A5C25730042616420636FB9
:107F80006D6D616E642E0A0052756E6E696E672E9D
:107F90002E2E0A00456E61626C696E6720696E74F0
:107FA000657272757074732E2E2E0A0064696E6984
:107FB000740064696F63746C0066696E697400664E
:107FC0006C6F6164006665786563006D636C656104
:107FD00072006D636F7079006D64696666006D6430
:107FE000756D70006D6562006D6568006D65770088
:107FF00068696400686965006866640068666500B1
:1080000063616C6C006A6D70007265737461727488
:1080100000726573657400696E666F0074657374D1
:1080200000746261736963006D6261736963006B00
:10803000696C6F00656400FFAC7F00000102010005
:108040000000000000000000B27F000001040100F9
:108050000000000000000000B97F000001140300D0
:108060000000000000000000BF7F0000012B0300A3
:108070000000000000000000C57F00000130030088
:108080000000000000000000CB7F0000013C040065
:108090000000000000000000D27F0000013D04004D
:1080A0000000000000000000D87F0000013F040035
:1080B0000000000000000000DE7F0000014004001E
:1080C0000000000000000000E47F00000141040007
:1080D0000000000000000000E87F000001420400F2
:1080E0000000000000000000EC7F000001430400DD
:1080F0000000000000000000F07F000001500500BB
:108100000000000000000000F47F000001510500A5
:108110000000000000000000F87F0000015405008E
:108120000000000000000000FC7F00000155050079
:10813000000000000000000000800000017907003E
:10814000000000000000000005800000017807002A
:10815000000000000000000009800000018208000B
:1081600000000000000000001180000001830800F2
:1081700000000000000000001780000001850800DA
:1081800000000000000000001C80000001870800C3
:10819000000000000000000021800000018C0900A8
:1081A000000000000000000028800000018D090090
:1081B00000000000000000002F800000018E090078
:1081C000000000000000000034800000018F090062
:1081D000000000000000000000151915000100005B
:1081E000488702201200000000020000728702206F
:1081F0004300000000030000CC87022000000000C4
:10820000010309045A870220000000000203090448
:10821000B68702200000000003030904D087022073
:10822000000000000000000000000000000000004E
:10823000F8870220F8B500BFF8BC08BC9E4670471E
:0C824000217300001D050000DD6000003F
:04824C00F8B500BFC2
:108250000000000000C0022000000000FFFF070037
:1082600000000010FFFF010000000014FF0F0000DD
:108270000000FF1FFFFF03000000000000000000DF
:1082800000000000000E2707000E27070101010172
:10829000000000000000000001000000FFFFFFFFE1
:1082A0001201100102000040C01683047602010290
:1082B000030118035400650065006E007300790027
:1082C0006400750069006E006F000902430002013E
:1082D00000C0320904000001020201000524001060
:1082E00001052401010104240206052406000107FA
:1082F00005820310004009040100020A0000000783
:108300000503024000000705840240000000160338
:1083100055005300420020005300650072006900C0
:1083200061006C00040309040C030000000000005D
:1083300000000000000000000000000000000A042F
:1083400073670000736700007367000073670000C5
:1083500000000000E48A02204C8B0220B48B022033
:10836000000000000000000000000000000000000D
:1083700000000000000000000000000000000000FD
:1083800000000000000000000000000000000000ED
:1083900000000000000000000000000000000000DD
:1083A00000000000000000000000000000000000CD
:1083B00000000000000000000000000000000000BD
:1083C00000000000000000000000000000000000AD
:1083D000000000000000000000000000000000009D
:1083E000000000000000000000000000000000008D
:1083F000000000000000000001000000000000007C
:108400000E33CDAB34126DE6ECDE05000B00000040
:10841000000000000000000000000000000000005C
:10842000000000000000000000000000000000004C
:10843000000000000000000000000000000000003C
:10844000000000000000000000000000000000002C
:108770000000000000000000F88702200000000058
:1087800000000000248C0220248C02202C8C02206B
:108790002C8C0220348C0220348C02203C8C022051
:1087A0003C8C0220448C0220448C02204C8C022001
:1087B0004C8C0220548C0220548C02205C8C0220B1
:1087C0005C8C0220648C0220648C02206C8C022061
:1087D0006C8C0220748C0220748C02207C8C022011
:1087E0007C8C0220848C0220848C02208C8C0220C1
:1087F0008C8C0220948C0220948C02209C8C022071
:108800009C8C0220A48C0220A48C0220AC8C022020
:10881000AC8C0220B48C0220B48C0220BC8C0220D0
:10882000BC8C0220C48C0220C48C0220CC8C022080
:10883000CC8C0220D48C0220D48C0220DC8C022030
:10884000DC8C0220E48C0220E48C0220EC8C0220E0
:10885000EC8C0220F48C0220F48C0220FC8C022090
:10886000FC8C0220048D0220048D02200C8D02203D
:108870000C8D0220148D0220148D02201C8D0220EC
:108880001C8D0220248D0220248D02202C8D02209C
:108890002C8D0220348D0220348D02203C8D02204C
:1088A0003C8D0220448D0220448D02204C8D0220FC
:1088B0004C8D0220548D0220548D02205C8D0220AC
:1088C0005C8D0220648D0220648D02206C8D02205C
:1088D0006C8D0220748D0220748D02207C8D02200C
:1088E0007C8D0220848D0220848D02208C8D0220BC
:1088F0008C8D0220948D0220948D02209C8D02206C
:108900009C8D0220A48D0220A48D0220AC8D02201B
:10891000AC8D0220B48D0220B48D0220BC8D0220CB
:10892000BC8D0220C48D0220C48D0220CC8D02207B
:10893000CC8D0220D48D0220D48D0220DC8D02202B
:10894000DC8D0220E48D0220E48D0220EC8D0220DB
:10895000EC8D0220F48D0220F48D0220FC8D02208B
:10896000FC8D0220048E0220048E02200C8E022038
:108970000C8E0220148E0220148E02201C8E0220E7
:108980001C8E0220248E0220248E02202C8E022097
:108990002C8E0220348E0220348E02203C8E022047
:1089A0003C8E0220448E0220448E02204C8E0220F7
:1089B0004C8E0220548E0220548E02205C8E0220A7
:1089C0005C8E0220648E0220648E02206C8E022057
:1089D0006C8E0220748E0220748E02207C8E022007
:1089E0007C8E0220848E0220848E02208C8E0220B7
:1089F0008C8E0220948E0220948E02209C8E022067
:108A00009C8E0220A48E0220A48E0220AC8E022016
:108A1000AC8E0220B48E0220B48E0220BC8E0220C6
:108A2000BC8E0220C48E0220C48E0220CC8E022076
:108A3000CC8E0220D48E0220D48E0220DC8E022026
:108A4000DC8E0220E48E0220E48E0220EC8E0220D6
:108A5000EC8E0220F48E0220F48E0220FC8E022086
:108A6000FC8E0220048F0220048F02200C8F022033
:108A70000C8F0220148F0220148F02201C8F0220E2
:108A80001C8F0220248F0220248F02202C8F022092
:108A90002C8F0220348F0220348F02203C8F022042
:108AA0003C8F0220448F0220448F02204C8F0220F2
:108AB0004C8F0220548F0220548F02205C8F0220A2
:108AC0005C8F0220648F0220648F02206C8F022052
:108AD0006C8F0220748F0220748F02207C8F022002
:108AE0007C8F0220848F0220848F02208C8F0220B2
:108AF0008C8F0220948F0220948F02209C8F022062
:108B00009C8F0220A48F0220A48F0220AC8F022011
:108B1000AC8F0220B48F0220B48F0220BC8F0220C1
:108B2000BC8F0220C48F0220C48F0220CC8F022071
:108B3000CC8F0220D48F0220D48F0220DC8F022021
:108B4000DC8F0220E48F0220E48F0220EC8F0220D1
:108B5000EC8F0220F48F0220F48F0220FC8F022081
:108B6000FC8F022004900220049002200C9002202E
:108B70000C90022014900220149002201C900220DD
:0C8B80001C90022000000200FFFFFFFF1D
:00000001FF
